:100000000C94F9020C9416030C9416030C946212CF
:100010000C94BA360C9416030C948B360C94452928
:100020000C94F5310C94FE280C9416030C941603D2
:100030000C9478360C94ED280C9416030C9416034B
:100040000C9416030C9416030C9416030C941603CC
:100050000C9416030C9401370C9416030C9416039D
:100060000C9416030C9416034F0D510D530D550DA2
:10007000570D590D5B0D5D0D5F0D860D890D8C0DB6
:100080008F0D920D950D980D9B0D9E0D971E9A1E2E
:100090009D1EA01EA31EA61EA91EAC1EAF1EB21E34
:1000A00008200B200E201120142017201A201D20BC
:1000B000352038203B20412044203E2047204A2044
:1000C0004D2050208E209120942097209A209D2012
:1000D000A320A020A620C320C620C920CC20CF204A
:1000E000D220D520DB20D8200A210D211021132178
:1000F000162119211C211F212221252128212B21F4
:100100002E213522372239223B223D223F22412215
:10011000432245224722332205A84CCDB2D44EB902
:100120003836A9020C50B9918688083CA6AAAA2A9A
:10013000BE000000803F20446F6E65210065727232
:100140006F723A00416420696E66696E6974756DFC
:1001500000426C696E6B00556E6465726C696E6509
:100160000043572D520043570031202020487A0089
:1001700031302020487A0031303020487A00353044
:100180003020487A00312020206B487A003130201E
:10019000206B487A00313030206B487A00312020C3
:1001A000204D487A00313020204D487A0053706C41
:1001B00069740053706565642000524954200053EF
:1001C000656D690046756C6C00575350520043577B
:1001D000004F4646004F4E200052696E670054693A
:1001E000702000426F746800556C74696D617469A9
:1001F000630049414D42494320420049414D424933
:100200004320410053747261696768740053693513
:1002100033353141206572726F7200515250204C5B
:100220006162732C203230313900312E303100358B
:100230005720435720546376722000202F3D3F2ED5
:100240002C7E7F06DB07557365206F726967696EC8
:10025000616C204943210052657365742E2E2E2057
:1002600000204D487A0053656C6563742062616EAE
:10027000643A0053657474696E672075702E2E2E73
:1002800000C00DED146C1B8827C436C8461C524EA6
:1002900061746D0202020202020B0606060B0B02DB
:1002A0000302020003020300040107060101040126
:1002B00000030002020201010201010B0303070512
:1002C000030202020303030303030101010002030B
:1002D00002030003020200010301040101010403FF
:1002E000010002020002000002010B0B01070101E4
:1002F000065369676E616C2067656E2E00467265F5
:100300007175656E637900417564696F2043682E6D
:100310003200417564696F2043682E3100524620D7
:10032000506F77657200566F6C746167650050722C
:100330006573732053656C656374210047505320C7
:10034000646174610043616C20737973206F73631F
:100350000043616C20726566206F736300506861B2
:100360007365204869005068617365204C6F0049CF
:100370002D512062616C005065616B204250460037
:1003800053797374656D20667271005265662066DC
:10039000727100506861736520486920667271004F
:1003A0005068617365204C6F2066727100492D5151
:1003B0002062616C2066727100416C69676E206614
:1003C000727100537572653F20656E7465722031DD
:1003D0003700466163746F7279207273742E004324
:1003E0007573746F6D2073706C736800532D6D6539
:1003F00074657220737465700053686F7720532D95
:100400006D6574657200437572736F7220737479D1
:100410006C6500426174742E2073746570004261D3
:1004200074742E2066756C6C00426174742E207397
:10043000686F770044626C2E20636C69636B0053B5
:1004400065742074696D650057535052206C6F635A
:1004500061746F72005753505220706F776572004D
:10046000575350522063616C6C0053746172740076
:100470004672616D65004672657175656E637900DF
:100480004D6F646500426561636F6E00456E616229
:100490006C65206564697400456E61626C6520540A
:1004A0007800456E61626C6520527800416D706C19
:1004B0002E206176672E0053706565642061766733
:1004C0002E004E6F69736520626C6E6B2E00537444
:1004D00072676874206D6F64650053696465746F3A
:1004E0006E6520766F6C0053696465746F6E65206D
:1004F0006672710050726163746963650051534B99
:10050000004175746F205370616365004B657965B8
:100510007220576569676874004B6579657220734E
:10052000776170004B657965722073706565640052
:100530004B65796572206D6F6465004357206F6667
:1005400066736574004357206D6F646500524954AB
:100550002072617465005249540054756E652072B2
:100560006174650056464F20420056464F204100B8
:1005700056464F206D6F64650052657065617473F7
:1005800000496E74657276616C004D6573736167C6
:100590006520005072657365742000536176652094
:1005A00073657474696E6773210054657374206594
:1005B000717569706D656E7400416C69676E6D650B
:1005C0006E74004F7468657200426561636F6E00FF
:1005D0004465636F646572004B65796572005646C9
:1005E0004F004D6573736167657300507265736585
:1005F000740011241FBECFEFD8E0DEBFCDBF11E0E5
:10060000A0E0B1E0E6E0FFE702C005900D92A43F54
:10061000B107D9F725E0A4EFB1E001C01D92A630E3
:10062000B207E1F70E9450180C94813F0C9400002F
:1006300000C000C000C000C000C000C000C000C0BA
:10064000000008953C983D984498459808953C9A38
:1006500008953C9AEDDF1DD008953D9AE9DF3C985E
:10066000E7DF3D98E5DF3C9AE3DF13D00895082EDD
:100670003C9ADEDF802D0DD0882311F002D0F8CF18
:1006800008953D9A3C9AD4DF3D98D2DF3C98D0DF64
:1006900008950894881F01C0880F59F03D9A18F4F6
:1006A00000003C9802C03C9A00C0C2DF3D98C0DF09
:1006B000F3CF3D9A3C98BCDF3D98359BFECF882711
:1006C000349981E0B5DF99270895882701C081E03A
:1006D00071E03D9A3C98ACDF3D98AADF359BFECF98
:1006E000889434990894771FA0F73D9A813011F0CF
:1006F0003C9801C03C9A9CDF3D98359BFECF98DF2B
:10070000872F992708959091C503965081E09430E2
:1007100008F080E00895CF93C1E0C09322020E94C8
:1007200083038823D9F08FEF0E94D73680E00E94A0
:100730005F2C81E00E9414310E940C31809168008E
:100740008E7F8093680080917A00886080937A0021
:10075000C093700081E0CF910C948A328091C503E0
:100760008C3061F480E00E94ED3080E00E94143112
:1007700082E00E945210CF910C94D90F80E00E9429
:10078000ED3080E00E94143181E00E9452101092FE
:10079000800010926F00C09366048DEF80931D025D
:1007A00010921E0210921F0210922002109221023B
:1007B00080917A00877F80937A008091C5038B3087
:1007C00021F4C0938100CF91089587E08093810048
:1007D00081E0CF910C945F2C1092220280E00E9465
:1007E0005F2C80E00E9414310E946B108FEF0E94FA
:1007F000D736EAE7F0E080818860808381E08093EB
:10080000700080E00C948A32CF92DF92EF92FF92D8
:10081000CF938FE40E94811680916604882331F083
:1008200080911D028D3F11F083E001C080E20E94A3
:100830008E1680916604882309F4D3C02091640445
:10084000309165048091F4019091F501821793072E
:1008500050F46091640470916504681B790B6B011E
:10086000E12CF12C0DC0C0906404D0906504E12C03
:10087000F12C2FEFE21AF20AC81AD90AE108F1089E
:1008800080916404909165049093F5018093F40144
:1008900080E40E94811680911D0221E0280F8D3F87
:1008A00008F097C03091C5033A3049F4C11480E88C
:1008B000D806E104F10418F48FEFE81AF80A8091E1
:1008C0001E0290911F02A0912002B0912102BC0152
:1008D000CD016C0D7D1D8E1D9F1D60931E027093BA
:1008E0001F02809320029093210220931D023B302F
:1008F00061F430E040E050E00E94D23B69017A01AF
:100900008FECE81A8EEFF80A1AC0243039F46B0124
:100910007C0128E6E21A2EEFF20A11C030E040E036
:1009200050E00E94D23B69017A0186E6E80EF11C94
:1009300082E0CC0CDD1CEE1CFF1C8A95D1F74BE04D
:10094000C701B6010E941A388DE694E00E94A816ED
:1009500080911D02843009F044C086E391E00E943A
:10096000B416809168008E7F8093680081E0809348
:10097000700080E00E945F2C80E00E941431809122
:10098000C5038B3059F4C0921804D0921904E09238
:100990001A04F0921B040E944B1B0AC0C092E4038D
:1009A000D092E503E092E603F092E7030E94571B22
:1009B00080912B028823A9F00E94EC0310921D0461
:1009C00010922B0280E00E94CA0A83E08093DB042D
:1009D00008C020931D02CFE080E20E948E16C15015
:1009E000D9F78FEF80936604CF91FF90EF90DF905F
:1009F000CF9008950F931F938091570390915803C0
:100A000040911E0250911F026091200270912102BC
:100A1000480F591F611D711D40931E0250931F0204
:100A2000609320027093210280911D028F5F8931B3
:100A300019F080931D0248C010921D02E091F6014A
:100A400081E08E0F8A019B010E2E04C036952795FA
:100A5000179507950A94D2F7013311052105310541
:100A600028F0E82FEDCFEE2361F1E150DB01CA0160
:100A70000E2E04C0B695A795979587950A94D2F740
:100A800080319105A105B10570F3E093F6018093E3
:100A90001E0290931F02A0932002B09321020E9495
:100AA00021188EE00E9481168091F6010E949D1609
:100AB00010921E0210921F02109220021092210228
:100AC00003C01092F601E3CF1F910F910895109289
:100AD000DE031092170481E0809385020E94F813D0
:100AE0000C948B16CF931092300210922F0210921A
:100AF0002802109227028FEF90E0909326028093B5
:100B00002502809125048130A1F50E945539C82F16
:100B100080912D0490912E04A0912F04B091300467
:100B20006627782F892F9A2F27E731E040E050E0A1
:100B30000E94D23B2093AD033093AE034093AF03AA
:100B40005093B003CC2349F189EC95E00E94B41690
:100B500080E20E948E168DE391E00E94B41680E43C
:100B60000E9481168C2F0E9485208DE2809369045B
:100B700039C08091DE03882319F0809112040BC0E4
:100B800088EC90E09093CC038093CB038CE590E0CD
:100B90000E94563F862F0E946B138091DE038111C5
:100BA00007C08091FF0381110E948C290E94EE0CE6
:100BB00010922D02109223028FEF80932402109244
:100BC0002C028091370490913804A0913904B0919F
:100BD0003A048093A7039093A803A093A903B0932A
:100BE000AA03C0E08C2FCF91089591E09093DE038B
:100BF00090931704882319F09093BD0306C086E8EC
:100C000090E00E944E3F8093BD03109225040E9405
:100C1000720583E08093DB041092E90308958091CC
:100C20002C02811110C08091370490913804A0915A
:100C30003904B0913A048093A7039093A803A0933A
:100C4000A903B093AA0380912504813019F40E946E
:100C5000653B02C00E94AD06882311F18091DE033E
:100C6000882389F08091BD03882339F081508093D7
:100C7000BD03811102C00C94670588E890E00E94D2
:100C8000563F6093E9030E9472058091DE03811153
:100C900063C083E00E94521081E080932B0208958C
:100CA0004091A7035091A8036091A9037091AA03F2
:100CB0008091AD039091AE03A091AF03B091B003CA
:100CC000840F951FA61FB71F8093A7039093A803B7
:100CD000A093A903B093AA0380912504811107C0B2
:100CE0008091BA039091AB0389130E94CA1320919B
:100CF0002F02309130028091270290912802820FBA
:100D0000931F9093300280932F02209125023091FF
:100D1000260282179307D0F04091A7035091A803B1
:100D20006091A9037091AA034F5F5F4F6F4F7F4F90
:100D30004093A7035093A8036093A9037093AA0359
:100D4000821B930B9093300280932F028091DE03DD
:100D5000811102C00C947A0C089580912D028111AA
:100D60000DC080912302815080932302811109C01C
:100D700080912C02811105C082E001C081508093D6
:100D80002D02809123028F3F09F065C080912C02D3
:100D9000882379F020912C02215020932C0230914D
:100DA000F7013F3E09F03FC01092230210922E023D
:100DB00048C0909124029F5F909324022091CB031E
:100DC0003091CC03A901490F511DCA010E944E3F29
:100DD0008093F701811102C081E00895809123047E
:100DE0000E948E1F909124028917B1F38091F70120
:100DF0000E94031BE82FF0E0E85DFE4F2081209366
:100E0000F70187E030E09FEF980FA901082E02C09C
:100E1000559547950A94E2F740FF02C0892FF3CF1A
:100E200080932C02B7CF81E090E001C0880F2A9513
:100E3000EAF7832349F083E08093230281E08093E3
:100E40002E0210922A0207C081E080932302809331
:100E50002A0210922E0280912302811104C0109266
:100E60002A0210922E0280912A02811107C081E08D
:100E700090912E02911103C080E001C081E00E9498
:100E80000C1380E00895CF9380911604823079F09E
:100E90008091C5038D3F59F08C3F59F08091D30369
:100EA0009091D4038115904831F0C7E005C0CBE0A4
:100EB00003C0C9E001C0C0E080E48C0F0E9481162D
:100EC000EC2FF0E0E95CFD4F80810E948E1681E0FE
:100ED0008C0FCF91089580916A02A8E2B1E0E0E022
:100EE0009D91981719F0EF5FEA32D1F78EEF80935A
:100EF0006A02EA3010F480E303C0E43218F487E3B6
:100F00008E0F0895EA3229F0F0E0E95EFD4F8491FA
:100F100008958AE20895E7E3F2E080E2819392E0A7
:100F2000E734F907D9F708958091360290915E026F
:100F3000981779F08F5F803119F08093360202C0E4
:100F400010923602E0913602F0E0E559FD4F8081C3
:100F5000089580E008959091360280915E0298177E
:100F600099F09091360280915E02981779F0E7E34C
:100F7000F2E08181819382E0E734F807D1F70E94A3
:100F8000940780934602EDCF80E0089581E00895B4
:100F9000CF93DF93C82FD62F80911D048823D1F0E3
:100FA0008091BE03882351F18091BF03813051F4B9
:100FB000E0918602F0918702E359FB4FC0830E94C3
:100FC0007D281CC08230D1F48C2F0E94D53881112D
:100FD000EFCF14C080916802882381F080915E0277
:100FE0008F5F803119F080935E0202C010925E0222
:100FF000E0915E02F0E0E559FD4FC083DD2381F012
:1010000080916902882321F081E09091C60303C09A
:1010100081E09091D203911101C080E08093680239
:10102000DF91CF910895CF92DF92EF92FF9281E00E
:10103000809369022091120430E040E050E060EBC0
:1010400074E080E090E00E94D23B20935102309304
:1010500052024093530250935402A3E0B0E00E9426
:10106000103C6093560270935702809358029093FD
:101070005902DC01CB01820F931FA41FB51FB69547
:10108000A7959795879580934D0290934E02A093D4
:101090004F02B093500281E09091C603911101C0BC
:1010A00080E0809368028EEF80936A02109248027B
:1010B00010925502FF90EF90DF90CF90089510921C
:1010C000690208958F929F92AF92BF92CF92DF9262
:1010D000EF92FF9280917F0290918002A091810215
:1010E000B09182020496A11DB11D80937F0290935E
:1010F0008002A0938102B0938202E0905703F090A7
:1011000058038091C50387FD06C080916902811153
:1011100002C00E9413089091BA038091690299233A
:1011200029F0811141C00E9413083EC09091FC013A
:10113000992389F080917F0290918002A091810291
:10114000B09182028093F8019093F901A093FA0183
:10115000B093FB0129C0882339F180907F029090E1
:101160008002A0908102B09082028091F80190915B
:10117000F901A091FA01B091FB01881A990AAA0A13
:10118000BB0A20915102309152024091530250917A
:101190005402AEE0B0E00E94103C681579058A0563
:1011A0009B0510F4109269028091BA038093FC01B0
:1011B0004091690241113AC0E0910001F0910101B2
:1011C000EE15FF05F0F420910201309103016091CA
:1011D0001E042E153F0548F4C701821B930B70E0D7
:1011E0000E94BE3B260F371F08C0C9018E199F09F8
:1011F00070E00E94BE3B261B370B30930301209307
:10120000020180910201909103018E179F0720F443
:10121000F0930301E0930201809102019091030198
:10122000969587958E159F0520F481E08093630243
:1012300002C0109263028091630290915502891757
:1012400099F0C0907F02D0908002E0908102F090EF
:101250008202C0925A02D0925B02E0925C02F0924B
:101260005D02411124C025C0411121C0C0907F0200
:10127000D0908002E0908102F090820240915A0268
:1012800050915B0260915C0270915D02C41AD50AB4
:10129000E60AF70A4091E30350E060E070E04C1585
:1012A0005D056E057F0528F49091350289138093C2
:1012B00035022091350280914802281709F4F7C0C1
:1012C000C0907F02D0908002E0908102F090820274
:1012D00080915A0290915B02A0915C02B0915D02F4
:1012E000222311F18093490290934A02A0934B026A
:1012F000B0934C0280915F0290916002A0916102D4
:10130000B0916202C81AD90AEA0AFB0AC0926402C2
:10131000D0926502E0926602F09267028091FD0130
:10132000882309F48DC0C1C080935F02909360024E
:10133000A0936102B09362028091490290914A02A7
:10134000A0914B02B0914C02C81AD90AEA0AFB0AD2
:10135000C0923102D0923202E0923302F092340213
:10136000D701C6014E97A109B109873D9140A1055A
:10137000B10508F0E9C0E091CF03AE2FB0E01197BE
:1013800020914D0230914E0240914F0250915002F7
:101390000E941B3C6C0D7D1D8E1D9F1D2E2F30E06D
:1013A00040E050E00E94D23B20934D0230934E0229
:1013B00040934F0250935002E0911E04AE2FB0E0D4
:1013C0001197C216D306E406F506E8F420915102FF
:1013D0003091520240915302509154020E941B3CA2
:1013E0006C0D7D1D8E1D9F1D2E2F30E040E050E0C6
:1013F0000E94D23B209351023093520240935302F9
:1014000050935402A1C0209156023091570240914E
:101410005802509159020E941B3C6C0D7D1D8E1D7F
:101420009F1D2E2F30E040E050E00E94D23B2093E1
:10143000560230935702409358025093590284C089
:101440008090510290905202A0905302B0905402AA
:10145000A5E0B0E0A50194010E94103C6C157D054B
:101460008E059F0540F40E946B0760E00E94C8074C
:1014700061E080E218C08091560290915702A091DD
:101480005802B0915902880D991DAA1DBB1DB69531
:10149000A795979587958C159D05AE05BF0528F4F2
:1014A0000E946B0761E00E94C8071092FD018091C5
:1014B0003502811138C040917F02509180026091C5
:1014C00081027091820280915F0290916002A091EE
:1014D0006102B0916202481B590B6A0B7B0B809131
:1014E000560290915702A0915802B091590222E001
:1014F000880F991FAA1FBB1F2A95D1F7841795073C
:10150000A607B70780F48091FD0181110CC00E94ED
:101510006B0760E00E94C80761E080E20E94C80794
:1015200081E08093FD018091630280935502809158
:10153000350280934802FF90EF90DF90CF90BF90EC
:10154000AF909F908F900895409151025091520218
:10155000609153027091540280915602909157020B
:10156000A0915802B0915902480F591F6A1F7B1F62
:10157000769567955795479580916A02C416D5066A
:10158000E606F70610F4880F02C0880F8F5F80937D
:101590006A028BCFCF93C82F8091D603909183029C
:1015A000891B90918602890F0E948116CC2341F0FD
:1015B0008091DF03813011F48DE003C08EE001C023
:1015C0008CE0CF910C946B168091C5038D3F21F474
:1015D000809110048F5B08C09091100181E09230DF
:1015E00008F480E09F5F890F0E9481168EE00C94C2
:1015F0006B168091D3039091D40397FD12C08DE2B6
:101600000E948E162091D3033091D40380E090E89D
:10161000A0E0B0E0BC01CD01621B730B8109910910
:101620000FC08BE20E948E166091D3037091D40399
:10163000CB01A0E0B0E0BC01CD0170588109910957
:1016400046E00E941A388DE694E00C94A81680E4D7
:101650000E9481168AEB91E00E94B4160E94F90A5A
:101660000E947E160E94C3160C94E40A80E40E9435
:10167000811683EB91E00E94B41660E08091120421
:101680000E9413170E947E160C94C3164BE00E9412
:101690001A3880916D04803319F480E280936D04D0
:1016A000109276048DE694E00C94A816CF92DF9207
:1016B000EF92FF92CF93DF93C82FD62F69017A0163
:1016C0000E948116D11102C084E001C085E00E9411
:1016D0008E16C701B6010E94460B8091E203882353
:1016E00091F0C11110C08091E103811103C080E22B
:1016F0000E948E1680E5DF91CF91FF90EF90DF90F2
:10170000CF900C948E16DF91CF91FF90EF90DF90E9
:10171000CF900895A0918802B0918902B7FF11C0BF
:10172000BF7028EA35E24AE050E00E94103C20E019
:1017300034E840E050E00E94D23B3093890220938D
:10174000880280911101883009F04AC08091C50358
:1017500081111AC080E40E94811660918802709104
:1017600089026B5F7F4F80E090E047E00E941A386B
:101770008EE280936F0480E28093720486E580930A
:1017800073041092740428C0813051F580E40E94E3
:101790008116A0918802B0918902A657BD4F9D0184
:1017A0000E94FA3B28E334E441E050E00E94D23B3F
:1017B000CA01B9016B5F7F4F8F4F9F4F46E00E9478
:1017C0001A388EE280936E0480E28093710487E57C
:1017D00080937204109273048DE694E00C94A81622
:1017E000409121045091220426E0249FC001259FAE
:1017F000900D112420910404309105048217930761
:1018000018F4281B390B02C020E030E060918802F8
:101810007091890280E02617370730F4873021F075
:10182000240F351F8F5FF7CF9091FE01981721F09D
:101830008093FE010C944117089580911604823024
:10184000C9F42091EC033091ED034091EE035091E7
:10185000EF0360E080E00E94560B2091C7033091B7
:10186000C8034091C9035091CA0361E080E40E941B
:10187000560B2AC081110AC02091EC033091ED0370
:101880004091EE035091EF0360E00AC02091C7033E
:101890003091C8034091C9035091CA0361E080E0D0
:1018A0000E94560B80E20E948E168091D303909185
:1018B000D4038115904841F080E40E9481160E9473
:1018C000F90A80E20E948E1680911104882339F073
:1018D0000E948A0B8FE00E94811686E004C08FE090
:1018E0000E94811680E20E948E160E94E40A1092E5
:1018F0008502089580E40E9481168CE00E946B1698
:1019000080912504813031F580912C02813011F5D0
:1019100047E050E068EE73E08DE694E00E943E3FC1
:101920008DE694E00E94A81680E20E948E1645E0A3
:1019300050E06FEE73E08DE694E00E943E3F8DE64E
:1019400094E00E94A81680E20E948E168091DB032C
:101950000C949D16089580916D04882319F08130B0
:1019600021F0089586E691E002C081E691E00C94B2
:10197000B41680916D04882319F0813021F0089508
:1019800087E591E002C081E591E00C94B416809166
:101990006D04882319F0813021F0089584EC91E0E2
:1019A00002C08FEB91E00C94B41680916D048823F3
:1019B00019F085ED91E002C081ED91E00C94B41630
:1019C00080916D04882319F0813021F008958EEC08
:1019D00091E002C089EC91E00C94B41680E00E9482
:1019E000811660910C0470910D0480910E04909109
:1019F0000F044BE00E941A388DE694E00E94A8166E
:101A000080E20E948E168091250480936D040E94CE
:101A1000E00C80912504811107C080E20E948E169F
:101A2000809112040C949D1680E20C948E16809185
:101A30006D04813049F028F0823049F0833051F054
:101A4000089584E092E008C08BEF91E005C082EF3A
:101A500091E002C088EE91E00C94B41680916D0480
:101A6000813039F018F0823039F0089583EE91E03A
:101A700005C08EED91E002C089ED91E00C94B416A2
:101A800080E40E948116E0916D048E2F90E08930F1
:101A90009105C0F4FC01EC5CFF4F0C94F43B80E535
:101AA0000FC08CE30DC088E20BC08EE109C084E159
:101AB00007C081E105C08FE003C08CE001C08AE06F
:101AC0000E949D168DE60C948E1680916D048130D7
:101AD00051F038F0823051F48DEA91E00E94B41652
:101AE00005C081E401C082E40E948E160E947E1629
:101AF0000C94C316E0916D048E2F90E0893091050F
:101B000008F5FC01E35CFF4F0C94F43B85EA91E09F
:101B100017C08DE991E014C085E991E011C08DE80E
:101B200091E00EC085E891E00BC08EE791E008C01F
:101B300087E791E005C080E791E002C089E691E087
:101B40000C94B416089580916D04811105C084E44D
:101B500091E00E94B41603C060E00E9413170E9437
:101B60007E160C94C3160E94941F80916D048823E6
:101B700041F010927D048DE694E00E94A81680E06A
:101B8000089581E008950F931F93CF93DF9380E42E
:101B90000E9481168091BF0381114DC08091110177
:101BA000823061F48091C503811103C00E94650DEC
:101BB0003AC08630B1F40E94AB0C35C08330C9F412
:101BC0008091C503853019F40E94C70C2CC0811187
:101BD00003C00E94170D27C0893029F50E942E0DE1
:101BE00022C0833019F40E947A0D1DC08530D9F4CB
:101BF000FACF813039F48091C5038D30A1F40E9471
:101C0000A30D11C0853039F48091C503813059F49A
:101C10000E94E00C08C0863031F48091C503843006
:101C200011F40E94B90C0E947E16DF91CF911F9192
:101C30000F910C94C316833031F4DF91CF911F9133
:101C40000F910C94D50CC0918302D0918402C3599A
:101C5000DB4F00E110E08991882329F00E948E1665
:101C600001501109C1F7DF91CF911F910F91089594
:101C700081E0809385020895CF92DF92EF92FF92E8
:101C8000C0900401D0900501E0900601F09007019A
:101C9000209108013091090140910A0150910B01F6
:101CA000C701B6010E94333E20910C0130910D0115
:101CB00040910E0150910F010E949A3C20E030E0CB
:101CC00040E05FE30E94243C0E940C3D072E000C84
:101CD000880B990B0E94443D2AED3FE049EC50E40B
:101CE0000E94333EA70196010E949A3C6B017C0141
:101CF0000E94A03E60934E0370934F038093500365
:101D000090935103C701B6010E94953C6093520322
:101D10007093530380935403909355039B01AC013C
:101D20000E94243C60934A0370934B0380934C03BE
:101D300090934D03FF90EF90DF90CF9008952F92F6
:101D40003F924F925F926F927F928F929F92AF924B
:101D5000BF92CF92DF92EF92FF920F931F93CF9398
:101D6000DF9300D000D01F92CDB7DEB740900401C2
:101D7000509005016090060170900701C0904A03E1
:101D8000D0904B03E0904C03F0904D031982812CCE
:101D9000912CA12CB12C212C312C00E010E0282F0B
:101DA00030E03B832A833981232F30E03D832C832D
:101DB000B901330F880B990B0E94443DA301920196
:101DC0000E94903C87FF2BC0A7019601B101C8017A
:101DD0000E94333E9401A5010E94233C4B015C010B
:101DE0008C819D81EA81FB818E0F9F1F880F991F37
:101DF00086579D4FFC0160817181072E000C880B76
:101E0000990B0E94443DA50194010E94243CF98154
:101E1000FF5FF983410158011B018C01C4CF94017C
:101E2000A501B101C8010E94333EA70196010E949D
:101E3000333E6B017C019101A801B101C8010E94F0
:101E4000333E2B013C019401A501B401C5010E9460
:101E5000333E9B01AC01C301B2010E94243CA701A7
:101E600096010E94233C0E94AE3E0E94133D709357
:101E70005803609357030F900F900F900F900F909F
:101E8000DF91CF911F910F91FF90EF90DF90CF9056
:101E9000BF90AF909F908F907F906F905F904F908A
:101EA0003F902F90089590916D039F5F903119F0AE
:101EB00090936D0302C010926D03E0916D03F0E00A
:101EC000E35AFC4F80830895FA01D90111821082F0
:101ED0001C92813049F56330B9F040F4613071F003
:101EE000623009F044C02CE833E01AC0653091F04C
:101EF00070F06630E1F529E533E012C023E833E005
:101F00003183208396E032C022E733E005C02AE81F
:101F100033E006C020E933E0318320839FE026C010
:101F2000318320838C9323C0823029F46230F9F40A
:101F300025EA33E00DC0883029F46730C1F422EA85
:101F400033E011C0843099F4623031F42EE833E08C
:101F50003183208391E00AC0643048F063706330BD
:101F600031F42EE633E03183208392E09C9320818C
:101F70003181232B29F090918203892B8093820356
:101F800008950F931F93F9019081DB01A90FB11DF3
:101F90002C91281309C09F5F9083933031F4D801AE
:101FA0004C93108281E002C0108280E01F910F915B
:101FB000089580E40E9481168091820380FF05C00D
:101FC0008CE893E00E94A81603C08DE20E948E1652
:101FD00080E20E948E168091820381FF0FC0809163
:101FE000A503823319F482E591E00AC0833319F422
:101FF00085E591E005C088E591E002C08BE591E0C0
:102000000E94A81680E20E948E1686E60E948E1616
:102010008091820383FF10C08091A303811103C0CC
:1020200080E30E948E168091A2030E948E168091FA
:10203000A303882339F004C08DE20E948E168DE23E
:102040000E948E1680E20E948E1684E70E948E16F1
:1020500080917103909182039823A9F00E949D16AC
:1020600080E20E948E1683E70E948E1660917103B3
:1020700070E080915B0390915C030E94BE3B862FD1
:102080000E949D1604C08EE591E00E94A8160E9451
:102090007E16803520F480E20E948E16F8CF1092D2
:1020A000820308958093A0030E9472368091680095
:1020B00081608093680010926B008091A003813052
:1020C00031F480916B00806180936B00089583E50B
:1020D0009FE00C944E320E9446320E944B36109282
:1020E000A003E8E6F0E080818E7F808310926B0091
:1020F0000895CF93DF9300D000D01F92CDB7DEB705
:1021000080918C03813409F0ABC04091910350E081
:10211000405351092091900330E0205331096AE087
:10212000629FC001639F900D1124840F951F97FD3E
:1021300001969595879560915903653411F4865BF6
:1021400003C099E4981B892F898380917203E091E1
:102150008A03EE3411F4865E03C099E7981B892F39
:102160008A838091920390E0C0977AE0749F9001F7
:10217000759F300D1124820F931F97FD0196959541
:102180008795653431F46AE00E94B23B905D9B8391
:1021900006C06AE00E94B23B89E3891B8B83909161
:1021A0007303EE3411F49C8303C089E6891B8C838E
:1021B0001D82CE0101960E944039811126C045E062
:1021C00050E06FEE73E08DE694E00E943E3F99810F
:1021D00080916D0498130FC09A8180916E049813BA
:1021E0000AC09B8180916F04981305C09C818091E7
:1021F0007004981751F045E050E06FEE73E0CE01A7
:1022000001960E945C3F0E94553940918703440F1C
:102210004056842F880F880F480F80918803805381
:10222000480F60918503660F6056862F880F880FD0
:10223000680F809186038053680F80918303880F15
:102240008056982F990F990F890F9091840390537E
:10225000890F0E94212A8091290281110E948C29D4
:102260008091A003823019F40E94D90F09C08330F5
:1022700039F40E946B108AE08093C5030E948B039F
:102280000F900F900F900F900F90DF91CF910895C6
:102290000F931F93CF93C82F8091080281113DC0E7
:1022A000809107028C278093070208E012E026E065
:1022B00032E041E063E671E08C2F0E94C10F882379
:1022C00059F0109206021092050210920402109228
:1022D000030210920202DAC008E012E025E032E0C8
:1022E00042E067E671E08C2F0E94C10F8111E9CFB7
:1022F00024E032E048E06BE671E08C2F0E94C10FD1
:102300008111DFCF23E032E044E06FE671E08C2FF3
:102310000E94C10F8111D5CFB9C0C43249F41092C7
:102320000802109206021092020210920702AEC03A
:1023300020910202CC3219F0CA3209F059C08091C2
:10234000000290910102009769F0409106023091DD
:10235000FF01FC01431718F4E40FF11D02C0E30F65
:10236000F11D108280910802843061F5243050F113
:10237000822F8370833031F5273051F480918E03A2
:10238000813331F410925C0310925B03109271035D
:10239000E0910002F09101028081882399F08EE69D
:1023A00093E00E94E43820915B0330915C03620F5C
:1023B000731F70935C0360935B03809171038F5F65
:1023C00080937103609102026F5F6093020210922A
:1023D00006022FEF31E040E052E0809108020E94B7
:1023E000640FCA3211F48EEF11C0809107024BC006
:1023F0002E3F79F48C2F0E94DC389091070220E167
:10240000829F90191124909307028FEF809302020C
:102410003DC02F3FE1F48C2F0E94DC3890910702E1
:10242000981B909307021092020280910802992350
:1024300039F080959091820389238093820326C08E
:10244000813021F5CF911F910F910C94791020913B
:10245000000230910102809107022115310599F0A7
:10246000909106024091FF01941768F48C278093A5
:102470000702F901E90FF11DC083809106028F5F09
:102480008093060203C0C827C0930702CF911F9113
:102490000F9108958091A10390916D03891789F0A0
:1024A0008F5F803119F08093A10302C01092A103C5
:1024B000E091A103F0E0E35AFC4F80810E944811B3
:1024C000E9CF08951F920F920FB60F9211242F9308
:1024D0003F934F935F936F937F938F939F93AF93AC
:1024E000BF93EF93FF938091A003813069F48091B3
:1024F000840090918500909365048093640483B177
:1025000080718093660402C00E94E031FF91EF91D8
:10251000BF91AF919F918F917F916F915F914F91FB
:102520003F912F910F900FBE0F901F901895CF9352
:10253000C82F0E94DF1A882371F18091B703882386
:1025400051F1C11115C04091370450913804609188
:10255000390470913A0480910B0290910C02A09181
:102560000D02B0910E0284179507A607B70798F4DD
:1025700080E00E946A3280E00E94963280E00E94F1
:10258000ED3081E00E9490321092B70380916F008D
:102590008B7F80936F00CF910895CF92DF92EF925F
:1025A000FF922091E00360912D0470912E048091A0
:1025B0002F0490913004C0903704D0903804E090FC
:1025C0003904F0903A04222381F02091120430E083
:1025D00040E050E00E94D23BA0E6B0E00E94103CF8
:1025E0002AE030E040E050E004C024E630E040E083
:1025F00050E00E94D23BC20ED31EE41EF51EC092D4
:102600000B02D0920C02E0920D02F0920E02FF90AB
:10261000EF90DF90CF900895CF93C82F0E946A3239
:102620000E94DF1A811114C080911101883081F05D
:10263000C093B703CC2311F080E001C081E00E9479
:10264000903280E00E94963280E00E94ED3039C0E6
:10265000CC2379F180E00E9490328091B703811100
:102660000AC08091E203811103C081E00E94ED3035
:1026700081E08093B7038091E203811103C081E080
:102680000E9496328091CD03811104C0809117047D
:10269000882361F08FEF9FEFDC0180930B02909312
:1026A0000C02A0930D02B0930E020BC00E94CD123B
:1026B00008C080910A0281110E94CD1280E00E9420
:1026C00096328091BA038093AB03C093BA03C09350
:1026D0000A02CF910895CF92DF92EF92FF920F936B
:1026E0001F93282F30E040E050E060912D0470915E
:1026F0002E0480912F04909130040E94D23BACE0D4
:10270000B0E00E94103C2AE030E040E050E00E943F
:10271000D23BCA01B9012093AD033093AE0340937D
:10272000AF035093B0032091140430911504690154
:10273000E12CF12C243F314068F41092B20304EFF5
:1027400011E020E030E0A90198012C193D094E0963
:102750005F0909C021E02093B203A7019601245F1D
:102760003140410951090E94A23B28EE33E040E08C
:1027700050E00E94D23B2093B3033093B4034093C4
:10278000B5035093B6031F910F91FF90EF90DF9028
:10279000CF9008950F931F939091B2034091A70398
:1027A0005091A8036091A9037091AA030091B3030B
:1027B0001091B4032091B5033091B603882339F00A
:1027C000992339F0400F511F621F731F06C09923D0
:1027D000C9F3401B510B620B730B4093A70350933B
:1027E000A8036093A9037093AA031F910F91089502
:1027F000809112040E946B138091370490913804E9
:10280000A0913904B0913A048093A7039093A80350
:10281000A093A903B093AA0380910704811103C078
:1028200082E08093AC0308954F925F926F927F9203
:102830008F929F92AF92BF92CF92DF92EF92FF92D0
:102840000F931F93CF93509107048091AD03909104
:10285000AE03A091AF03B091B0030091A703109114
:10286000A8032091A9033091AA035523F9F04091C0
:10287000AC034423D9F01092AC034091B9034770E4
:10288000A9F4AC01BD01440F551F661F771FD90184
:10289000C801840F951FA61FB71F8093A7039093AD
:1028A000A803A093A903B093AA03C1C0C0903704A2
:1028B000D0903804E0903904F0903A0426013701B2
:1028C000401A510A620A730A4C015D01880C991C76
:1028D000AA1CBB1C84149504A604B70428F48C0D10
:1028E0009D1DAE1DBF1D04C0800F911FA21FB31FF1
:1028F0008093A7039093A803A093A903B093AA037E
:1029000051110EC08091AC03813051F48091B90314
:10291000877019F01092AC0303C082E08093AC037F
:10292000809109028823F1F081508093090281117E
:102930007EC00E940C138091B9038C7F8093B903F1
:10294000809109020E94CA1381E08093AC038091B8
:10295000CD03813009F06BC08091B903877E8093ED
:10296000B90365C09091CD038091B903913041F4D2
:10297000282F28742834D1F0282F2073203359F0C1
:1029800082FF18C02091B103213051F4933019F027
:1029900092E09093B10393E0909309028B7D2DC058
:1029A000933019F091E09093B10391E09093090274
:1029B0008B7B17C080FD0FC081FF07C093E0909311
:1029C000090292E09093B10317C09230C1F4282F0E
:1029D0002874283441F491E09093B1039093090254
:1029E0008F7B80620DC0282F2073203341F4909399
:1029F000B10393E0909309028F7D806401C08F79C9
:102A00008093B9038091B903877E8093B903809145
:102A100009020E940C13C0910902CC2319F08C2FDB
:102A20000E94CA1381E0C11180E08093B803CF9166
:102A30001F910F91FF90EF90DF90CF90BF90AF90DC
:102A40009F908F907F906F905F904F900895CF925E
:102A5000DF92EF92FF92CF938091DE038111BDC090
:102A6000809117048111B9C0809122028111B5C0F3
:102A70000E94DF1A811104C08091C50387FDADC09B
:102A80000E940734C82F0E941F342091CD032111CA
:102A900010C0C11106C091E0811101C090E0892FE2
:102AA00001C081E0CF91FF90EF90DF90CF900C9428
:102AB0000C13C0903704D0903804E0903904F090A3
:102AC0003A044091A7035091A8036091A903709123
:102AD000AA034C155D056E057F0510F030E008C0B7
:102AE0009091AC03992319F091E09093B80331E0F1
:102AF000C1110CC081111EC0223051F18091B90367
:102B0000887F8093B9031092B1033FC09091B903BD
:102B1000882319F09C7F946024C091FF19C09C7F8A
:102B200094609093B903233009F451C092E09093DC
:102B3000B1034DC09091B90390FF0AC09C7F94608F
:102B40009093B9032330E1F081E08093B10318C082
:102B50009091B803992381F0CC2331F09091B9037F
:102B600091609093B90333C0882379F08091B903C1
:102B700082608093B90304C0C11129C0882329F061
:102B80008091B90380618093B90331110E941414BC
:102B900080910704811121C08091AC038230E9F457
:102BA0008091B9038770C9F01092AC03809137040B
:102BB00090913804A0913904B0913A048093A7030E
:102BC0009093A803A093A903B093AA0306C0909181
:102BD000B90398609093B903D1CFCF91FF90EF9054
:102BE000DF90CF9008955C9A00C05C9808950F9391
:102BF0001F9381E00091370410913804209139042B
:102C000030913A0440910F025091100260911102EC
:102C100070911202401751076207730708F080E0B5
:102C20001F910F910895CF93C82F0E94292A809158
:102C3000370490913804A0913904B0913A048C0F74
:102C4000911DA11DB11D80930F0290931002A093BE
:102C50001102B0931202CF9108951F93CF93DF9387
:102C6000D82F162F409137045091380460913904C1
:102C700070913A0480910F0290911002A09111027C
:102C8000B091120284179507A607B70718F00E94A3
:102C9000292AE8CFCBB1C07F8C2FD7FD8860D6FD25
:102CA0008460D5FD8260D4FD8160D3FDC860D2FD13
:102CB000C460D1FDC260D0FDC1608BB9112311F099
:102CC000449A01C044980E94F315CBB9DF91CF918B
:102CD0001F910C94F315CF93C82F60E00E942D161E
:102CE000C43010F487E201C082E0CF910C94131637
:102CF00061E00E942D1682E00C9413168091BB03B4
:102D00000895CF93C82F80E88C0F0E946B16C09354
:102D1000BB03CF91089581E00C946B1661E00E9493
:102D20002D1682E00E9413168091BB038F5F809363
:102D3000BB030895805D0C948E16CF936AE00E94C9
:102D4000B23BC92F0E949A168C2FCF910C949A16E1
:102D5000CF93DF93EC018991882319F00E948E169E
:102D6000FACFDF91CF910895CF93DF93FC01849147
:102D7000EF012196882321F00E948E16FE01F7CFE5
:102D8000DF91CF910895CF93C82F8091BB03C817CF
:102D900019F08C2F0E948116C03140F48091BB0342
:102DA000803160F480E20E948E16F8CF8091BB03E0
:102DB000803520F480E20E948E16F8CFCF910895DE
:102DC00080E70E946B1680E00E94781682E00E94E5
:102DD000781686E00E9478168EE00E9478168EE1C2
:102DE0000E9478168EE00E94781686E00E9478167F
:102DF00082E00E94781680E00E94781681E00E94AE
:102E0000781681E00E94781685E00E94781689E0A5
:102E10000E9478168FE10E94781688E00E9478164A
:102E200084E00C9478160F931F93CF93DF93D62FE3
:102E3000082F10E0843640F0CCE9C80FC43638F0D3
:102E4000C8E3C80F82E004C0C82F80E001C081E061
:102E50000436110510F00E949A1680E090E0CA3006
:102E600018F0CA500196FBCF0A30110508F4D111B1
:102E70000E949A168C2FDF91CF911F910F910C9485
:102E80009A16CF93DF93D82F80E70E946B168EE0BF
:102E90000E947816C6E0DC1710F08FE101C081E1D6
:102EA0000E947816C150B9F78FE1DF91CF910C9451
:102EB0007816CF93DF933C9A549A509A519A529A2B
:102EC000539A80E49CE90197F1F7599A589A0E9425
:102ED000F31580E891E60197F1F70E94F315C0E43D
:102EE000D1E0CE010197F1F70E94F315CE010197D1
:102EF000F1F758980E94F3152197F1F788E20E94A4
:102F00006B1688E00E946B160E948B1686E00E946A
:102F10006B168CE00E946B1680E0DF91CF910C94D1
:102F20004117CF9380E40E946B16C8E080E10E94B5
:102F30007816C150D9F7C23010F084E101C080E1A9
:102F40000E947816CF5FC830B1F7C0E0C23010F0F1
:102F500085E101C080E10E947816CF5FC830B1F7EB
:102F600080E00E9478168AE00E9478168FE10E9425
:102F700078168FE10E9478168FE10E9478168EE015
:102F80000E94781684E00E94781680E00E947816ED
:102F90008CE00E94781682E10E9478168EE10E94F1
:102FA000781682E10E94781682E10E94781680E00D
:102FB0000E94781680E00E94781680E00E947816C1
:102FC0008CE10E94781682E10E9478168CE10E94C2
:102FD000781682E10E9478168CE10E94781680E0D3
:102FE0000E94781680E00E94781680E0CF910C94C1
:102FF0007816611103C08BE00C94811670E061506B
:103000007109962F990F690F262F30E0F90132963A
:10301000482F50E0E417F50714F482E00FC068175A
:1030200010F080E20BC02F5F3F4F4217530711F49F
:1030300080E004C0E417F50719F481E00C948E16C3
:103040000895FF920F931F93CF93DF93F82E80E4A0
:103050000E948116C2E0D0E00F2D10E0C017D1070A
:1030600014F482E011C08C2F82508F1510F080E292
:103070000BC0CE0101970817190711F480E004C0B6
:103080000C171D0719F481E00E948E162396C23397
:10309000D10521F7DF91CF911F910F91FF900895F6
:1030A00085E085BD0E9452360E9459170E948B16FA
:1030B0000E94281B0E943C0E0E948B0781E00E9408
:1030C0009032789480E480937C008FEE80937A0035
:1030D00085EF93E00E944E3FC82F811109C08FE217
:1030E00092E00E94B4168AE292E00E94B41605C0F3
:1030F0008AE00E94B30D8111F2CF80E40E94811614
:10310000C11105C08BE192E00E94B41605C08BE0AE
:103110000E94B30D8111F6CF84E180936A048091FF
:103120006A04882359F080E00E9429398091600068
:103130008111FCCF80916A048150EFCF0E94391D2C
:103140000E948B160E94911786EC90E00E944E3FE1
:10315000893018F00E943B1C03C082E08093DB049E
:10316000912CD0E0612CC0E0C12CD12C760100E084
:10317000B12CA12C4AE0842E77247A948091C50347
:103180008B3F51F480913B04682D0E94B23B80FF3D
:1031900002C0599A01C059988091DB04882309F430
:1031A00051C00E948B16911009C08DE092E00E94E0
:1031B000B41680E00E94ED300E948B167092C50319
:1031C0008091DB04813021F08091DB04823019F59D
:1031D00080E00E9490329091DB0481E0923009F00F
:1031E00080E00E94391D0E94CC290E94F81381E0E2
:1031F00080934C048093550480911704882321F018
:103200000E947205B82E15C080E00E9414310E9401
:10321000380EB12C0EC080911704882339F08091AC
:10322000DE03811103C00E94EE0C02C00E94380E22
:1032300004E10E945F0881E00E9490321092DB045A
:103240009924939480912902811129C080911704B7
:10325000882329F18091C5038F3F09F540913704F8
:10326000509138046091390470913A048091A70319
:103270009091A803A091A903B091AA038417950780
:10328000A607B70760F48091DE03882321F08091C0
:10329000E903811104C0B11002C00E940F068091A1
:1032A000C5038F3F49F480911704882329F080914A
:1032B000DE03882309F4CAC080915603803321F0CD
:1032C0008091560381117BC080916902811104C0F5
:1032D000809156030E949F0E80911101873059F40E
:1032E00080912202882339F00E948303882319F0F9
:1032F0000E94FA0402C00E94620880911101883085
:1033000099F58091C5038250823070F58091570302
:1033100090915803C80ED91EE11CF11CCF5FC03438
:1033200011F0C11111C0C701B60136E0969587951D
:10333000779567953A95D1F747E00E941A38C0E033
:10334000C12CD12C76013BC0C13021F480E40E9415
:10335000811635C0C83098F5EC2FF0E0E559FB4FE9
:1033600080810E948E162BC00E94DF1A882339F1BB
:103370008091E103882319F18091570390915803BC
:10338000C80ED91EE11CF11CCF5FC03111F0C11174
:1033900016C0C701B60124E0969587957795679585
:1033A0002A95D1F72091DC033091DD0340E050E015
:1033B0000E94D23B69017A01622ED0E0C0E00E94F7
:1033C000DF1A882399F0D63088F401110FC00E94CB
:1033D000F7158823D9F1D53029F06D2F862D0E945D
:1033E000F91702C00E94E40ADF5F30C00E94DF1AB2
:1033F000882361F18091D203811104C08091C603BA
:10340000882321F10E94F715882399F0002389F081
:10341000003158F411E0100FE02FF0E0E95CFD4FAF
:1034200080810E948E16012F11C00E94E40A00E0E4
:103430000DC00E94F715882349F0011107C00E94B2
:10344000AB07882319F00E944307082F0E94292AFE
:1034500080911C04811103C08091700080FF0E9444
:10346000D1330E94B332809166048F3F11F00E94E5
:1034700004040E944A128091690481110CC00E94C8
:10348000A332182FA81641F080916C04811104C05A
:103490000E94643401C01A2D0E9427368091450491
:1034A000882341F08091DB04811104C0109245040F
:1034B0000E941431809188029091890297FD0E94A8
:1034C0008A0B8091DE03882359F00E9407348823F9
:1034D00019F00E94670504C00E941F348111F9CFC2
:1034E00080911704882359F08091DE03811107C071
:1034F0008091800086FF03C080E00E946A320E94B3
:10350000271580E00E9497128091DC04882349F1FE
:1035100080FF0FC08091C5038F3F59F4809117043D
:10352000882339F0B11005C08091290281110E94D1
:10353000A1298091DC0481FF12C0109229028091A0
:10354000370490913804A0913904B0913A048093E3
:10355000A7039093A803A093A903B093AA03109282
:10356000DC048091EB0381110E94A02180918502EF
:10357000811106C080915E04811102C0A12EFECD92
:1035800080918502882319F00E941D0C02C00E94C0
:10359000E40A10925E048091C5038F3F11F0D6E0DB
:1035A000EDCF0023E1F38091D203811104C080911B
:1035B000C6038823A1F30E944307082FF0CF809110
:1035C000C5038F3F39F094E0980F81E0923018F0F6
:1035D00080E0089581E00895883080F490E0FC0157
:1035E000EE0FFF1F8E0F9F1FFC01E258FE4F8081E0
:1035F0009181A281BC018A2F90E0089561E070E082
:1036000080E090E00895CF93882389F0C82F0E942E
:103610000C38843269F4EBE3F2E080E09491C9174E
:1036200021F08F5F31968B30C9F78C5D01C080E04F
:10363000CF9108958A3010F4805D0895843210F49B
:10364000895C0895E82FF0E0E95EFD4F84910895CC
:1036500084E090E00E94563FDC01CB01BF778132CD
:103660009D4CAB45B74071F080E790E00E94563F1B
:10367000673672418B4E9C4D29F086E492E00E94A1
:10368000B416FFCF089590E00296880F991F880F17
:10369000991F0C94563F4091180450911904609161
:1036A0001A0470911B0488E590E00C94743F4091DB
:1036B000E4035091E5036091E6037091E70384E52C
:1036C00090E00C94743F6091160483E090E00E94B7
:1036D000663F4091EC035091ED036091EE037091D1
:1036E000EF038CE790E00E94743F4091C703509134
:1036F000C8036091C9037091CA0380E890E00E94FA
:10370000743F6091100184E890E00E94663F6091F0
:10371000100485E890E00E94663F4091D3035091E9
:10372000D40360E070E088E490E00E94743F409130
:10373000120450E060E070E08CE590E00E94743F7D
:1037400040910004509101046091020470910304BF
:1037500080EC90E00C94743F83E090E00E944E3F38
:10376000809316048CE790E00E94563F6093EC0330
:103770007093ED038093EE039093EF0380E890E065
:103780000E94563F6093C7037093C8038093C90398
:103790009093CA0384E890E00E944E3F809310010A
:1037A00088E490E00E94563F7093D4036093D30363
:1037B00085E890E00E944E3F809310048CE590E0F5
:1037C0000E94563F6093120480EC90E00E94563FA6
:1037D00060930004709301048093020490930304A7
:1037E0000895CF92DF92EF92FF92CF93DF93E09113
:1037F0006D04F0E0EE0FFF1FEF57FD4F2591349160
:10380000A8EEB3E00E94FA3B6B017C01C8E0D0E077
:10381000B701A601CE010E94743F2496C834D10599
:10382000B9F7B701A6018CE790E00E94743FB70199
:10383000A60180E890E00E94743FB701A60184E7EA
:1038400090E00E94743FB701A60184EA90E00E94D4
:10385000743FB701A60180EC90E00E94743F609134
:103860006D0486EC90E0DF91CF91FF90EF90DF90B8
:10387000CF900C94663F8BEF8093C5030E948B160C
:1038800086E692E00E94B41610926D040E94400DEC
:103890001092DB040895CF93DF93EC010E948B1606
:1038A000CE010E94B416C0E0D0E060E0CE010E94DC
:1038B000663F2196C11584E0D807B9F747E652E183
:1038C0006BEE7CED80E790E00E94743F4CEB52E0A1
:1038D00060E070E080E590E00E94743F40E65CE0CC
:1038E0006CE971E084E590E00E94743F40E05DE2A5
:1038F00061E371E088E590E00E94743F4CE050E0A5
:1039000060E070E08CE590E00E94743F44EF51E08D
:1039100060E070E08CE690E00E94743F4CEB52E077
:1039200060E070E084EB90E00E94743F43E650E07A
:1039300060E070E088E790E00E94743F45E250E06C
:1039400060E070E088E690E00E94743F40E050E85C
:1039500060E070E088E490E00E94743F66E084E8F4
:1039600090E00E94663F67E085E890E00E94663F35
:1039700061E08CE990E00E94663F61E08DE990E0B3
:103980000E94663F61E08EE990E00E94663F4CEB4A
:1039900052E060E070E088EA90E00E94743F48E501
:1039A00052E060E070E08CEA90E00E94743F40E2F8
:1039B00053E060E070E080EB90E00E94743F40EEE6
:1039C0005EE260E070E088EB90E00E94743F48EEB9
:1039D00053E060E070E08CEB90E00E94743F4CE2BA
:1039E00051E060E070E080EA90E00E94743F4AE0BD
:1039F00050E060E070E080E990E00E94743F47E0B2
:103A000050E060E070E084E990E00E94743F4CE395
:103A100050E060E070E088E990E00E94743F44E686
:103A200050E060E070E08CE890E00E94743F6FEF3F
:103A300086EC90E00E94663F43E25DEC6BE577E048
:103A400084E090E0DF91CF910C94743F84E090E0AB
:103A50000E94563FDC01CB01BF7783329D4CAB45C2
:103A6000B74031F083E792E00E944B1C0C948B1618
:103A70000895CF93DF93C82F0E94261DC1110E9485
:103A8000AC1B84E590E00E94563F6093E403709382
:103A9000E5038093E6039093E70388E590E00E94B6
:103AA000563F609318047093190480931A049093FE
:103AB0001B048FE490E00E944E3F8093E00380E57A
:103AC00090E00E94563F609308047093090480932D
:103AD0000A0490930B0481E090E00E944E3F809393
:103AE000F80382E090E00E944E3F8093CD0384EF84
:103AF00093E00E944E3F8093F9038EE490E00E9491
:103B00004E3F8093BC038CE690E00E94563FEB0151
:103B100070931504609314048CE490E00E944E3F6F
:103B2000809317048DE490E00E944E3F809325041B
:103B300080E690E00E94563F6093FF0384E690E0A9
:103B40000E94563F6093D50388E690E00E94563F5E
:103B50006093DB0384E790E00E94563F60930C047F
:103B600070930D0480930E0490930F0486E890E008
:103B70000E944E3F8093BD0387E890E00E944E3F35
:103B80008093E2038FE990E00E944E3F80931104FE
:103B900088EB90E00E94563F709305046093040404
:103BA0008CEB90E00E94563F7093220460932104B6
:103BB00080EA90E00E94563F7093FD036093FC03FF
:103BC00080E990E00E94563F6093E30384E990E02F
:103BD0000E94563F6093CF0388E990E00E94563FD1
:103BE00060931E048CE990E00E944E3F8093D203C4
:103BF0008DE990E00E944E3F8093C6038EE990E0ED
:103C00000E944E3F8093BE0384EC90E00E944E3FA2
:103C10008093DF0385EC90E00E944E3F8093E103A8
:103C20008CE890E00E94563F7093DD036093DC03C4
:103C300087EC90E00E944E3F80930704E29730F4B7
:103C400082E390E09093150480931404809114040F
:103C500090911504873B934030F086EB93E090936E
:103C600015048093140489E08093810084EB90E034
:103C70000E94563F6E3581E0780710F46EE571E0E2
:103C80009B0140E050E0609118047091190480910C
:103C90001A0490911B040E94D23B30938900209318
:103CA00088008091880090918900969587959093DF
:103CB0008B0080938A0088E790E00E94563F83E65D
:103CC000861B8823A9F020918A0030918B004091B7
:103CD0008A0050918B0094E0569547959A95E1F7AC
:103CE000241B350B30938B0020938A008150E9CF41
:103CF00080911104811110923C04DF91CF910895BD
:103D0000E0911101EB3028F4F0E0ED58FE4F808196
:103D1000089580E00895E091C5038E2F90E08A30E9
:103D2000910520F5FC01EA5BFF4F0C94F43B8BEE10
:103D300095E01AC082EE95E017C08EED95E014C0B4
:103D400088ED95E011C080ED95E00EC089EC95E01E
:103D50000BC083EC95E008C089EB95E005C08AEACA
:103D600095E002C08BE995E00C94B416089580911B
:103D70001101853029F481E09091C503983009F054
:103D800080E00895CF92DF92EF92FF920F931F93FE
:103D90008091CB039091CC030E94563F209111015A
:103DA000223059F52091C503243039F5611520E8FA
:103DB00072078105910588F400E010E820E030E00A
:103DC00068017901C61AD70AE80AF90AC701B601DB
:103DD00047E00E941A388DE207C0705881099109A6
:103DE00047E00E941A388BE280936D041F910F9177
:103DF000FF90EF90DF90CF9008954091E8031F91DE
:103E00000F91FF90EF90DF90CF900C941A38EF92C3
:103E1000FF920F931F93CF93DF938C01EB017A01F5
:103E20000E94B71E882311F1809132042AE0622F8C
:103E30000E94B23B805D80936D04905D90936E0410
:103E40008AE380936F0480913D040E94B23B805DC1
:103E500080937004905D909371041092720486E0D8
:103E60008093E80382E08093BF032DC08091C50357
:103E700090E0F701E80FF91F24912093BF03FE01A2
:103E8000E80FF91FC491C093E803880F991FD80168
:103E9000A80FB91F8D919C919093CC038093CB0375
:103EA000223019F40E94C21E0EC0213041F44C2F62
:103EB00050E0BC018DE694E00E943E3F04C00E94A9
:103EC0004E3F80936D04DF91CF911F910F91FF9032
:103ED000EF900C94C30D83E995E00E94B416809195
:103EE000C50360E08F5F0E94131782E08093BF03D9
:103EF0008BE08093E8038091C50390E00296880FE1
:103F0000991F880F991F9093CC038093CB030E9435
:103F1000563F4BE00E941A380C94C30D843010F0C9
:103F200082E3089584E60895843010F042E301C0EE
:103F300044E64093E803843038F424E6829FC001CD
:103F4000112488539F4F0BC090E0049752E3589F71
:103F50009001599F300D1124C901885A9D4F9093AB
:103F6000CC038093CB0350E06091CB037091CC03E2
:103F70008DE694E00C943E3F8091C5038C3099F41B
:103F800081E895E00E94B41682E08093BF0383E04D
:103F90008093E80388E890E09093CC038093CB0370
:103FA0000E94C21E27C08D30A1F489E795E00E94CF
:103FB000B4161092BF0381E08093E80386E890E096
:103FC0009093CC038093CB030E944E3F80936D046B
:103FD00011C08AE895E00E94B4168091C50360E0A4
:103FE0008F5F0E94131781E08093BF038091C50308
:103FF0000E94941F0C94C30DE091C5038E2F90E096
:1040000088309105F0F4FC01E05BFF4F0C94F43B29
:1040100080E795E014C08AE695E011C084E695E05B
:104020000EC08AE595E00BC086E595E008C08DE4FA
:1040300095E005C085E495E002C08BE395E00E9421
:10404000B41641EE52E069EE72E084EE91E00C9419
:10405000071FE091C5038E2F90E08A30910520F56F
:10406000FC01E85AFF4F0C94F43B80E395E01AC042
:1040700084E295E017C089E195E014C08DEF94E0EB
:1040800011C08CE095E00EC081E095E00BC084EF9C
:1040900094E008C087EE94E005C08AED94E002C089
:1040A0008EEC94E00E94B4164DEC52E067ED72E0A5
:1040B00080ED91E00C94071F8091C503823099F048
:1040C00038F4882369F08130C1F487EB94E013C0A1
:1040D000843079F058F0853081F48CE894E00BC09E
:1040E00082EC94E008C08CEA94E005C082EA94E097
:1040F00002C088E994E00E94B41641EC52E067ECFB
:1041000072E084EC91E00C94071F90E089309105F7
:1041100008F5FC01EE59FF4F0C94F43B85E894E060
:1041200017C080E894E014C086E794E011C080E7EF
:1041300094E00EC08AE694E00BC080E694E008C0EC
:1041400085E594E005C088E494E002C08FE394E044
:104150000C94B41608958091C5030E94852041EB0C
:1041600052E069EB72E084EB91E00C94071FE09160
:10417000C5038E2F90E08930910508F5FC01E559C3
:10418000FF4F0C94F43B84E394E017C089E294E081
:1041900014C08EE194E011C083E194E00EC086E08B
:1041A00094E00BC089EF93E008C08CEE93E005C06B
:1041B00082ED93E002C08FED93E00E94B4168091EF
:1041C000C503883099F480E40E94811683EC93E063
:1041D0000E94B41682E08093BF0383E08093E803DB
:1041E00043E060E070E0CB010C941A384FE952E0F4
:1041F00068EA72E082EA91E00C94071FE091C5033F
:104200008E2F90E08D30910568F5FC01EC58FF4F42
:104210000C94F43B89EB93E023C08DEA93E020C03B
:1042200080EA93E01DC083E993E01AC08BE893E035
:1042300017C080E893E014C087E793E011C08FE6D1
:1042400093E00EC086E693E00BC08DE593E008C0D6
:1042500081E593E005C085E493E002C08CE393E040
:104260000E94B41680912202882349F08091C503F0
:10427000863018F40E94EC0302C00E948B038091E8
:10428000C503863040F443E952E069E972E086E90B
:1042900091E00C94071F80912202811107C080E4F5
:1042A0000E9481168EE293E00C94B4160895CF928A
:1042B000DF92EF92FF92CF93C1E0C0931C04C090B5
:1042C0001804D0901904E0901A04F0901B04C70160
:1042D000B60120E03AE040E050E00E94D23B30934B
:1042E000D1032093D003C701B6012AE030E040E0BB
:1042F00050E00E94D23B209324042093B3001092FC
:10430000F00310928500109284001092EB03EAE70C
:10431000F0E08081877F8083C0936F0010928100DE
:10432000C093B1001092B2008FEF9FEF90932004E2
:1043300080931F04CF91FF90EF90DF90CF9008956E
:1043400080E40E9481162091D7033091D8034091D8
:10435000D9035091DA03AAE0B0E00E94103C4AE091
:104360000E941A38EDE6F4E08EE28183868185832F
:10437000878186831782CF010E94A81681E692E08A
:104380000E94B4160C94572110926F00EAE7F0E0F7
:1043900080818860808310921C0408958FEF0E94B2
:1043A000D7368091C5038230B1F028F4882349F0D4
:1043B000813051F008958430A9F080F08530C1F04B
:1043C000089586E293E002C08DE193E00E94B41666
:1043D00010923C04089582E193E002C087E093E0EC
:1043E0000C94B4168DEF92E00E94B4160C945721F1
:1043F00081EF92E00E94B41682E08093BF0380ECCC
:1044000090E09093CC038093CB038CE08093E803FF
:104410000E94C21E0C94C30D0E948B168091110144
:104420008A3031F08F5F0E949A168EE20E948E16BB
:10443000909111018091C5039A3011F4893039F0BF
:1044400060E08F5F0E94131780E20E948E16E09159
:1044500011018E2F90E08B309105C8F4FC01EF57CD
:10446000FF4F0C94F43B0C948B1E0C946B1F0C941C
:10447000BC1F0C94FC1F0C9429200C945C200C9401
:10448000AB200C94B7200C94FE200C94CE21089500
:10449000E0918602F0918702E359FB4F80818B32D5
:1044A00011F48DE201C08BE2808308958091BF03F7
:1044B0008330E1F080911101823029F49091C5039D
:1044C000963069F413C08330B9F49091C5039923F1
:1044D00059F1993069F081E09530A9F425C099230C
:1044E00019F1933039F0953071F404C081E00895EA
:1044F00082E0089588E00895853039F481E0909154
:10450000C503913089F080E00895813031F48091C5
:10451000C5038D30C1F783E608958630A1F781E0A9
:104520009091C503943079F70895809111018830F6
:1045300059F48091C503833019F48FEF0C94D7366A
:10454000843011F40C94C42108958DE694E00E9407
:10455000E438609300047093010480930204909304
:10456000030482E00C941431CF92DF92EF92FF9219
:104570000F931F93CF93DF93E82E082F10E0E801ED
:10458000C359DB4F8881893341F50E94B71E8111E1
:1045900022C0E11002C0F12C24C0FF24FA94FE0CCA
:1045A000CF2CD12CFF2051F0F601E359FB4F808135
:1045B0000E94D538811102C0FA94F2CFF601E35976
:1045C000FB4F80810E94D538882329F38F2D0E94CC
:1045D000B422882301F380E301C08F5F8883FF2426
:1045E000F39480918602909187020817190779F059
:1045F0000E947E1690E0005C1F4F8017910721F00B
:1046000080E48E0D0E94811688810E948E168F2D67
:10461000DF91CF911F910F91FF90EF90DF90CF909E
:104620000895CF92DF92EF92FF920F931F93CF9353
:10463000DF93E82E082F10E0E801C359DB4F888193
:10464000803341F50E94B71E811122C0E11002C0E3
:10465000F12C24C0FF24FA94FE0CCF2CD12CFF2087
:1046600051F0F601E359FB4F80810E94D53881114A
:1046700002C0FA94F2CFF601E359FB4F80810E9409
:10468000D538882329F38F2D0E941123882301F325
:1046900089E301C081508883FF24F39480918602CE
:1046A000909187020817190779F00E947E1690E012
:1046B000005C1F4F8017910721F080E48E0D0E944F
:1046C000811688810E948E168F2DDF91CF911F91C8
:1046D0000F91FF90EF90DF90CF90089580916D043F
:1046E000811102C084E007C09091C503843040F47A
:1046F000933021F487E080936D04089588E0FBCF28
:10470000933011F4883071F30895CF93DF93809143
:104710001D04882309F4A3C080E00E94CA0A809186
:10472000BF03813009F477C028F08230E1F0833094
:1047300009F090C080916D04811103C00E9456223F
:1047400001C0815080936D0480911101823041F449
:104750008091C503853011F0833011F40E946E23DF
:104760000E94C30D77C080911101823069F480915D
:10477000C503843049F48091860290918702892B89
:1047800019F40E94482204C0809186020E941123DD
:104790000E94B71E8823C9F080916D04893319F4F3
:1047A00082E380936D0480916D04823339F48091AB
:1047B0006E04843318F083E380936E048091700458
:1047C000893319F485E3809370040E947E1640912A
:1047D000860250918702282F30E0CA01805C9F4FEB
:1047E0002817390721F080E4840F0E948116E09198
:1047F0008602F0918702E359FB4F80810E948E165A
:1048000080911101883031F58091C503853011F513
:104810000E94A5221FC0E0918602F0918702E35911
:10482000FB4F80810E94031B811101C08FE2C09168
:104830008602D091870281500E941A1BC359DB4F18
:104840008883E0918602F0918702E359FB4F8081D3
:104850000E948E1681E0DF91CF910C94CA0A0E94CB
:10486000801E9091C503981798F40E94952280911C
:10487000C503811104C00E94801E8093C5038091EE
:10488000C50381508093C503DF91CF910C940C2216
:10489000DF91CF910895CF93DF9380911D048823FA
:1048A00009F4A4C080E00E94CA0A8091BF0381304D
:1048B00009F478C028F08230E9F0833009F091C023
:1048C000C0916D04CF5FC0936D040E9456228C1777
:1048D00010F410926D0480911101823041F48091A6
:1048E000C503853011F0833011F40E946E230E94BD
:1048F000C30D77C080911101823069F48091C503A6
:10490000843049F48091860290918702892B19F4B2
:104910000E94482204C0809186020E94B4220E9414
:10492000B71E8823C9F080916D04833319F480E3A6
:1049300080936D0480916D04823339F480916E040C
:10494000843318F080E380936E0480917004863382
:1049500019F480E3809370040E947E1640918602D1
:1049600050918702282F30E0CA01805C9F4F2817A2
:10497000390721F080E4840F0E948116E0918602BD
:10498000F0918702E359FB4F80810E948E1680913F
:104990001101883031F58091C503853011F50E94F1
:1049A000A5221FC0E0918602F0918702E359FB4FD8
:1049B00080810E94031B8F5F8F3208F080E0C091DE
:1049C0008602D09187020E941A1BC359DB4F88834D
:1049D000E0918602F0918702E359FB4F80810E94AB
:1049E0008E1681E0DF91CF910C94CA0A80E00E947C
:1049F000CA0A0E949522C091C503CF5FC093C50328
:104A00000E94801EC81710F01092C503DF91CF914D
:104A10000C940C22CF93DF938091BF03813009F077
:104A20007AC08091860290918702FC01E359FB4F86
:104A300020812F3759F521E0280F3091E803231703
:104A400048F4A22FB0E0A359BB4F4C9111974C935F
:104A50002F5FF5CF009799F02081211110C00197A9
:104A600090938702809386028091830290918402C2
:104A7000009729F001979093840280938302E0913C
:104A80008602F0918702E359FB4F1DC02E37F9F4DF
:104A9000209106042083A091E8034FEF4A0F242FB2
:104AA00030E08217930748F423593B4FE9012197DF
:104AB0005881E90158834150F2CF80E28083B0E011
:104AC000A459BB4F1C9280818093060422C02630DB
:104AD000A1F4109287021092860210928402109222
:104AE000830210926D041092060480E40E948116E5
:104AF0000E947E160E94C3160CC0273061F480917C
:104B0000060480838091E80390E09093870280936D
:104B1000860281E001C080E0DF91CF910895CF92BD
:104B2000DF92EF92FF920F931F938091BF0381302A
:104B300081F4E0918602F0918702E359FB4F808176
:104B400092E8980F923018F08650823010F40E944C
:104B50000A25109287021092860210928402109207
:104B6000830210921D040E94911780E00E94CA0ADD
:104B70000E94C30D0E94B71E8823E1F0609170046B
:104B8000660F6056862F880F880F680F809171041A
:104B90008053680F80916D04880F8056982F990F6D
:104BA000990F890F90916E04905340E0890F0E94F5
:104BB000212A61C02091BF03223009F049C08091B1
:104BC00011018230F9F48091C5038430D9F48EE666
:104BD00094E00E94E43820916D042D3269F400E0E5
:104BE00010E820E030E068017901C61AD70AE80A27
:104BF000F90AB701A6010CC0AB01BC0150586F4FB8
:104C00007F4F06C08DE694E00E94E438AB01BC0102
:104C1000209111012630A9F42091C503283089F490
:104C20004131510561057105D1F587E592E00E949A
:104C30004B1C1F910F91FF90EF90DF90CF900C9441
:104C40003B1C8091CB039091CC030E94743F13C016
:104C50008091CB039091CC03213049F44091E8033B
:104C600050E0BC018DE694E00E945C3F04C060917E
:104C70006D040E94663F84E090E00E94563F97FDDD
:104C80000EC043E25DEC6BE577E884E090E01F91B5
:104C90000F91FF90EF90DF90CF900C94743F1F9195
:104CA0000F91FF90EF90DF90CF9008950E940A251A
:104CB000811149C02091BF038091860290918702A3
:104CC000213041F4FC01E359FB4F2081211102C046
:104CD00020E220830097E1F4E0918602F0918702C0
:104CE000E359FB4F8081809306042DC0809186029A
:104CF000909187020097A9F0FC01E359FB4F808156
:104D00000E94D53881110DC0809186029091870252
:104D1000019790938702809386028091BF0382302F
:104D200029F320918602309187028091830290912D
:104D300084022817390710F40197FBCF909384025F
:104D400080938302C9CF0E94C30D81E00C94CA0AEC
:104D5000CF93C82F0E940A25811144C02091BF0320
:104D600080918602909187022130C1F4FC01E359C1
:104D7000FB4F2081211112C020E220830FC0E0915F
:104D80008602F0918702E359FB4F80810E94D5385B
:104D900081110DC0809186029091870201969093B7
:104DA0008702809386028091BF03823041F3809115
:104DB0008602909187022091830230918402AC0197
:104DC000421B530B4031510518F02F5F3F4FF7CF77
:104DD0003093840220938302FC01E359FB4F8081CE
:104DE000809306048091E80390E0AC0141505109A2
:104DF00020918602309187022417350750F0CC238A
:104E000019F0CF910C948F2502979093870280938D
:104E100086028091BF039FEF980F923080F4E0915B
:104E20008602F0918702E359FB4F9081911107C0F0
:104E3000823011F480E301C080E280830AC0809157
:104E4000FE03882339F0E0918602F0918702E3594E
:104E5000FB4F11820E94C30D81E0CF910C94CA0ACE
:104E600080E40E94811683E50E948E1680E20E94F3
:104E70008E168091CE03893048F480E20E948E160F
:104E80008091CE038F5F0E949A1605C08091CE0359
:104E90008F5F0E949D1680E20E948E168091CE0345
:104EA0000E94431B0E94460B80E20E948E168CE4F7
:104EB0000C948E161F93CF93DF9380E40E9481168B
:104EC0008091230460E08F5F0E9413178EE20E949E
:104ED0008E1680E20E948E16809123040E94941FF9
:104EE000CDE6D4E01991111107C00E947E16DF9122
:104EF000CF911F910C94C3160E947E168035A8F79F
:104F0000812F0E948E16EECF20911004283078F465
:104F100030E0F901EE0FFF1F2E0F3F1FF901E2589D
:104F2000FE4F208131814281642FA90104C041E0FC
:104F300050E060E070E02091D3033091D4038823E7
:104F400039F0420F531F403187EA580768F408C010
:104F5000C901841B950BAC01413F98E5590720F02E
:104F60005093D4034093D3030E94270B81E0809396
:104F70004504089590911204882321F0933638F463
:104F80009F5F03C0923018F09150909312040E94DA
:104F9000360B0C94F81390916D04882331F09F5FC9
:104FA000993050F010926D0409C0911104C088E04E
:104FB00080936D0403C0915090936D040C94400D48
:104FC000882361F08091CE038F5F8093CE03809120
:104FD000CE03803171F41092CE030BC08091CE03CA
:104FE000882321F08091CE03815001C08FE080930F
:104FF000CE030C943027882361F0809123048F5FC7
:1050000080932304809123048C3071F41092230444
:105010000BC080912304882321F0809123048150C8
:1050200001C08BE0809323040C945A2780911604CE
:10503000813059F48091CE034091C7035091C80349
:105040006091C9037091CA030AC08091CE03409158
:10505000EC035091ED036091EE037091EF0390E04B
:105060000296880F991F880F991F0C94743F8091A6
:105070001604813069F48091CE030E94431B609333
:10508000C7037093C8038093C9039093CA030CC0ED
:105090008091CE030E94431B6093EC037093ED0359
:1050A0008093EE039093EF0381E080934C0480E0C3
:1050B0000C9414310E94952280911D04882319F0CC
:1050C0000E948F2514C0809111018A3051F0809385
:1050D000C5038AE0809311010E940C220E94EC0318
:1050E00006C081E08093DB048EE18093690480E058
:1050F0000E940C1380E00C94963280911D0488234A
:1051000019F081E00C94A826809111018A3071F485
:105110008091C503893021F40E94631B0C945A28A6
:10512000809311011092C5030C940C22873051F426
:105130008091C503863068F08091220281114CC0B5
:105140000C948B03883029F48091C503853009F0D5
:1051500043C08091BF03813039F490916D04911167
:1051600003C08093FE0304C01092FE03813011F44B
:105170000E94E0168091BF03823051F48091E803D1
:10518000833031F481E090E090938702809386022F
:1051900081E080931D0480E48093D6038091110107
:1051A000883059F48091C503853099F480E00E94DD
:1051B000903282E00E9414310CC0863051F480910C
:1051C000C503883031F40E94C30D0E947E160E94F0
:1051D000C31681E00C94CA0A08951F920F920FB66D
:1051E0000F9211248F938091F0038F5F8093F003CF
:1051F0008F910F900FBE0F901F9018951F920F92D6
:105200000FB60F9211242F933F934F935F936F9399
:105210007F938F939F93AF93BF93EF93FF9380916F
:105220001C048823F9F080911F04909120040196BA
:105230009093200480931F04892B19F487E08093B6
:10524000810020911F04309120048091D00390911F
:10525000D1032817390741F4809170008260809350
:10526000700002C00E94D133FF91EF91BF91AF91C6
:105270009F918F917F916F915F914F913F912F916E
:105280000F900FBE0F901F9018951F920F920FB6A0
:105290000F9211242F933F938F939F93AF93BF93BC
:1052A00080911C04882341F180911F049091200477
:1052B00001969093200480931F04892B11F0109283
:1052C000810020918400309185008091F00390E06E
:1052D000A0E0B0E0DC0199278827820F931FA11D71
:1052E000B11D8093D7039093D803A093D903B093B3
:1052F000DA0381E08093EB03809170008D7F8093CF
:105300007000BF91AF919F918F913F912F910F901E
:105310000FBE0F901F9018959091D50320913D04DA
:105320003091FF03892F281710F0830FFCCF809353
:105330002C048C3310F090932C0481E0809329028C
:10534000089580E40E948116809132040E949D1687
:105350008AE30E948E1680913D040E949D168AE386
:105360000E948E16809131040E949D1680E20E9458
:105370008E1680E20E948E168CE30E948E1680E2CA
:105380000E948E1680912C040E949D1680E20E943D
:105390008E1680E20C948E16CF92DF92EF92FF92DF
:1053A000CF93DF9316BC10923704109238041092FA
:1053B000390410923A046091180470911904809194
:1053C0001A0490911B046B017C012AE0F694E79487
:1053D000D794C7942A95D1F7C0922D04D0922E0469
:1053E000E0922F04F0923004EB01D370D0933F048D
:1053F000C0933E04C0923304D0923404E09235044A
:10540000F092360420E038EC40E050E00E94D23BBD
:10541000C20ED31EE41EF51EC0922604D0922704AD
:10542000E0922804F0922904D0932B04C0932A041C
:1054300087E2DF91CF91FF90EF90DF90CF900C94B7
:10544000131660933D0480933204409331040C940E
:10545000CC298F929F92AF92BF92CF92DF92EF9220
:10546000FF92CF93DF9396B58091130281112AC0EA
:1054700097FF3FC081E08093130280913C04882312
:1054800069F080911101883049F48091C503823020
:1054900028F480913C04815080933C0480916904FD
:1054A000882319F081508093690480913B048F5FB9
:1054B00080933B04809168048823D9F081508093C5
:1054C000680417C097FD15C010921302409137046D
:1054D000509138046091390470913A045F5F6F4FC6
:1054E0007F4F40933704509338046093390470938E
:1054F0003A04C0903704D0903804E0903904F0901A
:105500003A04CC24C90ED11CE11CF11CC092370412
:10551000D0923804E0923904F0923A048091260443
:1055200090912704A0912804B09129040097A10527
:10553000B10509F4B8C08C159D05AE05BF0508F08E
:10554000B2C01092670410923B0460912D047091D8
:105550002E0480912F0490913004C0912A04D091A0
:105560002B0420913E0430913F04C20FD31F809042
:10557000330490903404A0903504B0903604860E25
:10558000971EA81EB91E9E01232F33272695269508
:10559000820E931EA11CB11C80923304909234049D
:1055A000A0923504B092360422E330E040E050E0AF
:1055B0000E94D23BDA01C901880D991DAA1DBB1DAD
:1055C0008093260490932704A0932804B093290481
:1055D000D370D0932B04C0932A0481E088169104E1
:1055E000A1048FEFB806B0F08091A7039091A803B3
:1055F000A091A903B091AA038C199D09AE09BF0916
:105600008093A7039093A803A093A903B093AA0340
:105610000E94CC298091E903882319F0815080935E
:10562000E90380913C04882329F080913C04815057
:1056300080933C04809131048F5F8C3319F0809308
:10564000310416C01092310480913D048F5F8C3379
:1056500019F080933D040CC010923D0480913204F7
:105660008F5F883119F08093320402C010923204A7
:105670008091DC04982F91609093DC0420913D048C
:1056800090912C0429130FC090912902992359F06D
:1056900090912504992321F090913104992319F0D8
:1056A00083608093DC04DF91CF91FF90EF90DF90D7
:1056B000CF90BF90AF909F908F900895CF93DF933E
:1056C000D82FC62F80EC0E9437038D2F0E944903EC
:1056D000811109C08C2F0E944903811106C00E94CC
:1056E000410380E003C083E001C084E0DF91CF91FB
:1056F00008954F925F926F927F928F929F92AF9296
:10570000BF92CF92DF92EF92FF920F931F93CF93AE
:10571000C82F462E6701780149015A0187E0880C9D
:10572000991CAA1CBB1C8A95D1F7C501B401A7011D
:1057300096010E94D23BCA01B901512C612C712CF7
:1057400027E0440C551C661C771C2A95D1F722E0F3
:10575000521A61087108460E571E681E791EA7016D
:1057600096010E94A23B861A970AA80AB90A6D2DD3
:105770008C2F0E945E2B6C2D81E08C0F0E945E2B83
:10578000D301C20188279927A370BB27BD018827B1
:10579000992782E08C0F0E945E2B652D83E08C0F91
:1057A0000E945E2B642D84E08C0F0E945E2BCC2423
:1057B000DD248FE0E822FF244CE0F694E794D794B0
:1057C000C7944A95D1F7D501C40188279927AF70AE
:1057D000BB276C2D6A2B85E08C0F0E945E2B692DF8
:1057E00086E08C0F0E945E2B682D87E08C0FCF9196
:1057F0001F910F91FF90EF90DF90CF90BF90AF90EF
:105800009F908F907F906F905F904F900C945E2B45
:10581000CF92DF92EF92FF920F93CF93DF93C82F37
:10582000D22F4450510961097E4F6A017B0187E004
:10583000CC0CDD1CEE1CFF1C8A95D1F760E08C2F90
:105840000E945E2B61E081E08C0F0E945E2BD701ED
:10585000C60188279927A370BB276D2F602B6A2B61
:1058600082E08C0F0E945E2B6D2D83E08C0F0E94D6
:105870005E2B6C2D84E08C0F0E945E2B60E085E037
:105880008C0F0E945E2B60E086E08C0F0E945E2BE6
:1058900060E087E08C0FDF91CF910F91FF90EF9048
:1058A000DF90CF900C945E2BCF93C82F0E942203E1
:1058B00060E88C2F0E945E2BCF910C942703CF932E
:1058C000C82F0E942203CC2371F060E28CE30E9477
:1058D0005E2B60E48BEB0E945E2B63E482E10E940E
:1058E0005E2B60E008C060E08BEB0E945E2B82E1E3
:1058F0000E94542C64E083E00E945E2BCF910C94B4
:105900002703EF92FF920F931F93CF93C82F0E940C
:10591000220380914B048C17A8F5409144042C2F4E
:1059200030E090E04423C9F08901081B190BC8013D
:10593000092E000CAA0BBB0B40915104509152044C
:1059400060915304709154048A019B01081B190B48
:105950002A0B3B0BD901C80130C0A901481B590BC8
:10596000CA01092E000CAA0BBB0B409147045091B1
:1059700048046091490470914A04840F951FA61F42
:10598000B71F34C0C817D8F5409144042C2F30E01D
:1059900090E0821B930B092E000CAA0BBB0B442337
:1059A000A9F04091510450915204609153047091B8
:1059B0005404840F951FA61FB71F80935104909322
:1059C0005204A0935304B093540428C04091470458
:1059D000509148046091490470914A048A019B01E6
:1059E000081B190B2A0B3B0BD901C80180934704F4
:1059F00090934804A0934904B0934A040FC08C13B9
:105A00000DC06FE682E10E945E2BC0934B04CF91E4
:105A10001F910F91FF90EF900C942703E090510499
:105A2000F0905204009153041091540420914704C3
:105A3000309148044091490450914A0460914604D1
:105A400082E20E94792BDDCFCF92DF92EF92FF921C
:105A50009B01AC016091400470914104809142042B
:105A6000909143040E94A23B6093560470935704A4
:105A70008093580490935904C090E403D090E503B8
:105A8000E090E603F090E703A70196010E94D23B65
:105A900020934604462F572FBC018FEF9FEFAFE0B6
:105AA000B0E08093510490935204A0935304B093B8
:105AB000540424E180E090E0DC01440F551F661F90
:105AC000771F880F991FAA1FBB1F4C155D056E0518
:105AD0007F0528F04C195D096E097F09816021500E
:105AE00061F78093470490934804A0934904B093CE
:105AF0004A04FF90EF90DF90CF9008954F925F920D
:105B00006F927F928F929F92AF92BF92CF92DF92CD
:105B1000EF92FF920F931F93CF93DF93CDB7DEB732
:105B200028970FB6F894DEBF0FBECDBF29013A010A
:105B3000F50120914004309141044091420450917C
:105B40004304D6010E94103C4B015C01CF01A0E050
:105B5000B0E089839A83AB83BC83C801B701A501F8
:105B600094010E94D23B2D833E834F8358879B0133
:105B7000AC0169817A818B819C810E94A23BA50145
:105B800094010E94D23B49015A012D813E814F81EF
:105B9000588569817A818B819C810E94A23B950105
:105BA0008401060F171F281F391F009351041093FB
:105BB0005204209353043093540485E140E050E0B4
:105BC000BA01769567955795479540FE04C0400FFA
:105BD000511F621F731F76946794579447948150A6
:105BE00081F74093470450934804609349047093AD
:105BF0004A04411551056041710538F481E00115F1
:105C000011052041310508F080E028960FB6F89480
:105C1000DEBF0FBECDBFDF91CF911F910F91FF90DF
:105C2000EF90DF90CF90BF90AF909F908F907F903C
:105C30006F905F904F9008954F925F926F927F9216
:105C4000AF92BF92CF92DF92EF92FF920F931F938A
:105C5000CF93DF93CDB7DEB72D970FB6F894DEBFA5
:105C60000FBECDBF2B013C010E94220360E079EE04
:105C700084EA95E3A30192010E94D23B29833A83EF
:105C80004B835C83DA01C90181709927AA27BB275E
:105C900089879A87AB87BC8720FD03C0DA01C901D9
:105CA00007C089819A81AB81BC810197A109B109A3
:105CB0008093400490934104A0934204B093430422
:105CC0001D8660914004709141048091420490913E
:105CD0004304A30192010E94A23B61157644834CC8
:105CE000934208F46EC08D8581118EC0C301B2014C
:105CF0000E94242D8091470490914804A09149046A
:105D0000B0914A048D839E83AF83B887E090E4030B
:105D1000F090E5030091E6031091E703A12CBB246A
:105D2000B39457E7C52EDD24D3949C01AD01C30184
:105D3000B2010E947E2D882329F01092440491E044
:105D40009D87BFCF6091560470915704809158048D
:105D5000909159042091E4033091E5034091E603CA
:105D60005091E7030E94D23BA12CBB24B39437E7A8
:105D7000C32EDD24D3947B018C012D813E814F8184
:105D80005885C301B2010E947E2D882331F0A1E025
:105D9000A0934404B1E0BD8794CF809140049091DA
:105DA0004104A0914204B09143040297A109B109B2
:105DB0008093400490934104A0934204B093430421
:105DC00080CF9D85911120C089859A85AB85BC8542
:105DD000892B8A2B8B2B29F489819A81AB81BC81F9
:105DE00007C089819A81AB81BC810197A109B10962
:105DF0008093400490934104A0934204B0934304E1
:105E0000C301B2010E94242DE0905104F09052048D
:105E10000091530410915404209147043091480498
:105E20004091490450914A046091460482E20E94E4
:105E3000792B40914004509141046091420470914B
:105E4000430400E020E08AE30E94082C60EA81EB32
:105E50000E945E2B10924B042D960FB6F894DEBF75
:105E60000FBECDBFDF91CF911F910F91FF90EF90AB
:105E7000DF90CF90BF90AF907F906F905F904F90EA
:105E80000C9427033F924F925F926F927F928F9272
:105E90009F92AF92BF92CF92DF92EF92FF920F93B9
:105EA0001F93CF93DF93C82F6A017B01452B462BAD
:105EB000472B41F40E94542C81E0C13109F47BC18D
:105EC00080E079C14090E4035090E5036090E603E0
:105ED0007090E7030E94220380E8C81681EDD8067F
:105EE00080EFE80688E0F80608F07CC08091110198
:105EF0008830A9F485E08093C50360E079EE84EAF8
:105F000095E3A70196010E94D23B49015A01253829
:105F100033404105510508F03FC0312C5BC0C1142E
:105F200082E1D8068AE7E806F10408F41EC1C1142C
:105F30008BE1D80687EBE806F10408F41CC180EC7D
:105F4000C81681EED80684EEE806F10408F419C1FB
:105F500080ECC8168AEED80681E2E80681E0F806F1
:105F600008F415C180E8C81681EBD8068FE4E8066E
:105F700081E0F80608F411C180E8C8168AEBD8065B
:105F80008CE8E80681E0F80608F40DC18CE1882E63
:105F9000912CA12CB12C0CC107E0CC0CDD1CEE1C0B
:105FA000FF1C0A95D1F760E079EE84EA95E3A7013A
:105FB00096010E94D23B49015A01253833404105E0
:105FC000510530F014E8812E13E0912EA12CB12C54
:105FD000D0E73D2E80FE0DC081E0881A9108A1080F
:105FE000B10807C0B4E08B2E912CA12CB12CDCE0C1
:105FF000E0C0D0E0A7019601C501B4010E94A23B18
:10600000A30192010E94D23BE22FF4E120E030E0B4
:10601000A901660F771F881F991F220F331F441F86
:10602000551F641575058605970528F064197509CF
:10603000860997092160F15061F7CC24C39481EF60
:106040008E0F8C3458F0C12C60E88C2F0E945E2B90
:10605000C03109F086C060E881E181C0C03139F00B
:10606000AAE36A2EB0E2DB2E12E2712E05C07AE2BC
:10607000672ED12CFAE17F2EE0904D04F0904E0473
:1060800000914F04109150048091F8038E149F04E6
:10609000A006B10621F490911402981769F091E0DE
:1060A00090934C0480924D0490924E04A0924F0421
:1060B000B092500480931402EE24EA94FE2C0FE078
:1060C00010E06E2F872D0E94792B0D2F232DB50107
:1060D000A401862D0E94082CC031F1F4232DB501B6
:1060E000A40182E30E94082C60E085EA0E945E2BF6
:1060F000682D86EA0E945E2BCD2DCF646C2F80E147
:106100000E945E2B8091F803813019F46D2D6F652C
:1061100001C06C2F81E105C0C23129F46D2D6F647F
:1061200082E10E945E2B82E2781207C080914C04CB
:106130008823B9F060E881EB12C08AE1781211C0BF
:1061400080911001843020F080914C04882349F024
:1061500060E281EB0E945E2B10924C0402C00E9410
:106160005E2B0E9427038C2D26C05EE7852E912C86
:10617000A12CB12C1DC044E5842E912CA12CB12C56
:1061800017C030E4832E912CA12CB12C11C020E338
:10619000822E912CA12CB12C0BC098E2892E912C2F
:1061A000A12CB12C05C082E2882E912CA12CB12CFF
:1061B000D0E0312C1FCFDF91CF911F910F91FF9035
:1061C000EF90DF90CF90BF90AF909F908F907F9097
:1061D0006F905F904F903F900895CF93C82F0E948B
:1061E0002203CC2351F060E48BEB0E945E2B62E033
:1061F00083E00E945E2B63E409C060E08BEB0E94A9
:106200005E2B64E083E00E945E2B6FE480E10E94DD
:106210005E2BCF910C9427030E94220360E083E061
:106220000E945E2B0C942703CF92DF92EF92FF9295
:10623000CF93823071F44091000450910104609139
:1062400002047091030480E10E94422F8093550460
:10625000B1C0C091F803813009F044C084EA90E0F5
:106260000E94563F6B017C018091C503863059F432
:10627000409108045091090460910A0470910B0444
:10628000C130A1F41CC0883019F48CEA90E007C03A
:10629000893019F480EB90E002C088EA90E00E9417
:1062A000563FAB0160E070E0C13049F4D701C60150
:1062B000841B950BA60BB70BAC01BD0104C04C0DA4
:1062C0005D1D6E1D7F1D80E10E94422F809355044D
:1062D000B701A60182E1CF91FF90EF90DF90CF90C0
:1062E0000C94422F80911704882359F040910C049C
:1062F00050910D0460910E0470910F046A017B01AE
:1063000031C040911604411109C0C090EC03D090F7
:10631000ED03E090EE03F090EF030EC03091C70361
:106320002091C8039091C9038091CA03C32ED22E35
:10633000E92EF82E413071F4B701A60150586109D9
:1063400071098091D3039091D403480F591F611DA7
:10635000711D08C04091EC035091ED036091EE0374
:106360007091EF038091080490910904A0910A04B0
:10637000B0910B04C13029F4480F591F6A1F7B1FCD
:1063800004C0481B590B6A0B7B0B80E10E94422F13
:1063900080935504B701A60182E10E94422F8091AB
:1063A0005504811107C0CF91FF90EF90DF90CF90FF
:1063B0000C94380ECF91FF90EF90DF90CF9008951E
:1063C0001D9912C080916B008F7D80936B0080912E
:1063D000B200865A8093B40010925C04BA9A8091FD
:1063E000700084608093700008951F920F920FB622
:1063F0000F9211242F933F934F935F936F937F934B
:106400008F939F93AF93BF93EF93FF938091B200CD
:106410008F5B8093B40080915C04883090F480910D
:106420005C048F5F80935C0480915D04869580930B
:106430005D041D9B1AC080915D04806880935D049B
:1064400014C0809170008B7F80937000E0915A049B
:10645000F0915B04309719F080915D040995D89A0A
:1064600080916B00806280936B00FF91EF91BF91F0
:10647000AF919F918F917F916F915F914F913F91DC
:106480002F910F900FBE0F901F90189510927000D3
:10649000EBE6F0E080818F7D8083089521E42093F6
:1064A000B40090935B0480935A04E0E7F0E08081AD
:1064B0008B7F808383E08093B1002D9AE8E6F0E043
:1064C000808181608083D89AEBE6F0E080818062F1
:1064D00080830895882391F080911704882321F008
:1064E0008091DE03882351F0219A80E4809380001C
:1064F00080916F00846080936F000895219880914F
:106500006F008B7F80936F00809180008F7B8093E2
:1065100080000895882311F02B9A08952B980895F0
:10652000882311F0289A089528980895882311F057
:106530002A9A08952A98089589B186FB882780F9B8
:1065400091E08927089580916B0480FF02C084E068
:1065500001C080E090916B0491FD8E5F90916B047F
:1065600092FD8F5F0895CF92DF92EF92FF92CF93CB
:10657000DF939091C5039F3F39F4809117048823DE
:1065800019F080E88093120180911201803809F49B
:1065900001C138F08091120181508093120181E095
:1065A00006C0809112018F5F8093120180E09F3FAF
:1065B00009F06FC09091B7039111ECC090916B04FA
:1065C00090FF10C090911001811105C0933008F424
:1065D00058C0915004C0973008F053C09F5F90930B
:1065E00010014FC090911604913019F0CCEED3E019
:1065F00002C0C7ECD3E0811123C0C880D980EA80F3
:10660000FB80809110010E94EC1A6C157D058E05AF
:106610009F0588F4809110010E94EC1AC880D980EF
:10662000EA80FB80A7019601261B370B480B590B0C
:10663000DA01C9011FC0188219821A821B821EC08A
:10664000809110010E94EC1AC880D980EA80FB80FA
:10665000DC01CB018C0D9D1DAE1DBF1D811531EEE2
:10666000930735EFA30735E0B30720F08FEF90EEE7
:10667000A5EFB5E088839983AA83BB8381E08093EB
:106680004504DF91CF91FF90EF90DF90CF900C9475
:10669000380E9E3F41F4DF91CF91FF90EF90DF9055
:1066A000CF900C94E0279A3F41F4DF91CF91FF9077
:1066B000EF90DF90CF900C94FB279D3F29F59091B0
:1066C000B703911167C090916B0490FF15C0909132
:1066D0001004811104C0943038F0915003C09830F8
:1066E00018F49F5F90931004DF91CF91FF90EF908B
:1066F000DF90CF900C94E40ADF91CF91FF90EF9060
:10670000DF90CF900C9484279C3F41F4DF91CF9190
:10671000FF90EF90DF90CF900C94BA279B3F41F40D
:10672000DF91CF91FF90EF90DF90CF900C94CB272B
:1067300090911D049923E1F090916B0490FF18C093
:106740009091BF039150923098F4882349F080E0F3
:10675000DF91CF91FF90EF90DF90CF900C94A8261F
:10676000DF91CF91FF90EF90DF90CF900C94562661
:10677000882341F0DF91CF91FF90EF90DF90CF9091
:106780000C944B24DF91CF91FF90EF90DF90CF904E
:106790000C948523DF91CF91FF90EF90DF90CF9005
:1067A00008950E949C3229B1922F9095991F9927A4
:1067B000991F30911C02831304C030911B023917BA
:1067C00029F130911A02332329F030911B02391339
:1067D00010921A0230911A02311114C0882391F0DC
:1067E00030911C0231110EC031E030931A0227FDA6
:1067F00004C0209112012F5F03C02091120121508B
:106800002093120180931C0290931B0208958091A3
:10681000CD03811105C09091F903923078F409C03D
:106820008091BC03882329F083B185FB882780F9F8
:1068300003C083B18295817091E08927089583B167
:10684000807290911902891739F180931902809111
:1068500067048F3F21F08F5F809367041DC0809194
:10686000E203811119C08091DE03811115C080916E
:106870001704811111C08091220281110DC00E9464
:10688000DF1A811104C08091C50387FD05C081E036
:106890008093E2030E94380E8091CD03811105C0E0
:1068A0009091F9039D7F79F408C08091BC038823FF
:1068B00021F083B18295817004C083B185FB882764
:1068C00080F991E0892708950F931F93CF93DF9369
:1068D000D82F8091DE03811103C081E00E949712BE
:1068E0000E94A332C82F882329F08093180281E0E8
:1068F00080936C048091C5038C3F19F4D11164C15D
:1069000044C08D3F99F4D1115FC1C1FD41C0C0FFAA
:106910005BC180E090E89093D4038093D30383E03D
:106920008093DB0481E0809345044EC18B3F71F47A
:10693000CC2309F484C10E94F11B82E08093DB0424
:106940001092C5038AE0809311013EC18E3F79F415
:10695000D1113AC1C1FF03C00E94162819C0C0FF5F
:1069600003C00E94372814C0C2FF2EC111C08A3F45
:1069700099F4D11129C1C1FF02C080E003C0C2FF58
:1069800004C081E00E94F5051FC1CC2309F457C162
:1069900083E08093DB0418C187FD10C0D11114C1BE
:1069A00080911702811110C1C1FF03C00E947D2890
:1069B0000BC1C0FF09C10E945A2806C18091DE03A5
:1069C000811104C080911704882349F0C0FFFCC0E6
:1069D000809169048111F8C00E946705F5C0CC233D
:1069E00099F1D0911602D11128C0A091FC03B09169
:1069F000FD0320912D0430912E0440912F045091DD
:106A000030040E94103C28EE33E040E050E00E9449
:106A1000D23B8091370490913804A0913904B09111
:106A20003A04820F931FA41FB51F80935F049093B5
:106A30006004A0936104B0936204809117028111F5
:106A400003C0DF5FD0931602809116028230E1F01E
:106A500040915F0450916004609161047091620400
:106A600000913704109138042091390430913A0490
:106A7000401751076207730748F4CC2311F083E0F5
:106A800003C0882319F081E08093150280911502DC
:106A9000882309F499C09091180291FF19C083309E
:106AA00039F40E94801E8093C5030E944B247BC052
:106AB000823031F48DEF8093C5030E94270B73C0A1
:106AC000813031F48CEF8093C5030E94360B6BC08C
:106AD00020916804392F31702223C9F0332309F43F
:106AE0004AC08130A1F44091C7035091C80360911E
:106AF000C9037091CA034093EC035093ED03609374
:106B0000EE037093EF0393E09093DB042FC03323E5
:106B100091F1813089F4809116048F5F833018F4ED
:106B20008093160402C01092160483E08093DB0465
:106B300081E08093450437C0222309F44DC08230A0
:106B400009F052C08091EC039091ED03A091EE0307
:106B5000B091EF038093C7039093C803A093C90338
:106B6000B093CA0383E08093DB0481E08093450403
:106B70001092680418C092FF16C0813061F48091B1
:106B800010018F5F883008F084E08093100181E06D
:106B900080935E0408C08250823028F48AEF80938C
:106BA000C5030E945A2710921602109215028FEF09
:106BB0009FEFDC0180935F0490936004A0936104D5
:106BC000B093620410921802C0931702CC23C9F14B
:106BD00080E00E94293935C0823031F48EEF8093F5
:106BE000C5030E943027DFCF833029F64091EC03A4
:106BF0005091ED036091EE037091EF030091C70394
:106C00001091C8032091C9033091CA030093EC038B
:106C10001093ED032093EE033093EF034093C703EB
:106C20005093C8036093C9037093CA038093DB0435
:106C300081E0809345048CE480936804B4CF109283
:106C400017028C2FDF91CF911F910F9108958091A2
:106C50005F0490916004A0916104B091620440913E
:106C60003704509138046091390470913A048417C4
:106C70009507A607B70770F480E00E9464348FEF91
:106C80009FEFDC0180935F0490936004A093610404
:106C9000B0936204089586E08093B10081E0809310
:106CA000700008955E9A5F9A2C9A2D9A209A229AE3
:106CB000E8E6F0E0808182608083ECE6F0E08081AD
:106CC000886080838FEF9FEFDC0180935F04909357
:106CD0006004A0936104B093620480E00E946A3271
:106CE0000C944B36E0E7F0E080818E7F808308953E
:106CF0001F920F920FB60F9211248F93199B05C00C
:106D0000809182008068809382008F910F900FBEE7
:106D10000F901F9018951F920F920FB60F9211248B
:106D20002F933F934F935F936F937F938F939F9393
:106D3000AF93BF93EF93FF930E94333980916A041E
:106D4000811107C081E00E946434811102C0109259
:106D50006C04FF91EF91BF91AF919F918F917F91C3
:106D60006F915F914F913F912F910F900FBE0F90B8
:106D70001F9018951F920F920FB60F9211248F93A8
:106D80008FEE80937A0080917A0083FD05C0809118
:106D90007A00886080937A0080916B048061809390
:106DA0006B048F910F900FBE0F901F9018958F3F1F
:106DB000A9F480911101883021F48091C5038330BA
:106DC00051F080912202882341F081E09091C50327
:106DD000963019F403C081E001C080E020917C006E
:106DE0002F7030E0482F50E02417350749F090917C
:106DF0007C00907F890F80937C0081E08093630406
:106E000008951F920F920FB60F9211242F933F9364
:106E10004F935F936F937F938F939F93AF93BF93A2
:106E2000EF93FF9380916304882319F01092630419
:106E30007CC080917C008F70823069F480917800F2
:106E400090917900906890938902809388028FE0F6
:106E500080933C042CC080917C008F70833049F576
:106E600080916B04887F80936B048091780090916F
:106E70007900833D934020F080916B04816015C0C0
:106E800080917800909179008335934020F0809133
:106E90006B0484600AC08091780090917900853FEE
:106EA000914028F080916B04826080936B048FEF97
:106EB0003AC0E09156038091780090917900F0E01B
:106EC000EE0FFF1FE657FD4F91838083809156039D
:106ED0008F5F8093560380915603803611F4109291
:106EE000560380916B0484FF09C083E00E94D7366B
:106EF00080916B048F7E80936B0417C080913C045B
:106F0000811113C08091220281110FC08091110460
:106F1000811108C080911101883039F48091C50336
:106F2000823018F482E00E94D736FF91EF91BF9132
:106F3000AF919F918F917F916F915F914F913F9111
:106F40002F910F900FBE0F901F90189520E06115A4
:106F500071058105910539F060FD2F5F9695879544
:106F600077956795F4CF822F81700895262F269507
:106F700026952695820F911DFC01808190E070E09E
:106F8000609570956770772702C0959587956A958B
:106F9000E2F781700895262F269526952695FC0107
:106FA000E20FF11D70E0609570956770772721E022
:106FB00030E001C0220F6A95EAF78081282B2083F8
:106FC0000895262F26952695820F911DFC0180811C
:106FD00090E070E06095709563707727660F771F7B
:106FE00002C0959587956A95E2F783700895262FDC
:106FF00026952695FC01E20FF11D808170E06095D9
:10700000709563707727660F771F01C0440F6A95EC
:10701000EAF7482B4083089590ED980F9A3030F0AE
:107020009FEB980F9A3120F487530895892F089584
:1070300084E20895CF93C42F209111012230B9F436
:107040002091C503243099F461152AEC72072AE9CE
:1070500082072BE3920710F02DE201C02BE2209370
:107060006E0420E03AEC4AE95BE30E94D23B20E068
:10707000611531EE730735EF830735E0930728F08C
:10708000715E854F95402F5FF3CF205D20936F0495
:1070900020E0603836E9730738E98307910530F05E
:1070A00060587649884991092F5FF3CF205D20937E
:1070B000700420E0603432E473073FE083079105F9
:1070C00030F0605472448F4091092F5FF3CF205D00
:1070D000209371042CE22093720420E0603A36E899
:1070E000730731E08307910530F0605A764881409C
:1070F00091092F5FF3CF205D2093730420E060316E
:1071000037E273078105910530F0605177428109BC
:1071100091092F5FF4CF205D2093740420E0683E36
:1071200033E073078105910530F0685E7340810993
:1071300091092F5FF4CF205D209375042CE22093FA
:10714000760420E0643671058105910530F06456BF
:107150007109810991092F5FF5CF205D2093770494
:1071600020E06A3071058105910530F06A5071099F
:10717000810991092F5FF5CF205D20937804605D30
:107180006093790410927A04EEE0F0E0EC1BF109D0
:10719000E359FB4FADE6B4E080E08C1721F091910C
:1071A0009D938F5FFACFCF91089590ED980F81E076
:1071B0009A3008F080E0089590ED980F9A3010F022
:1071C00087530895892F08958F929F92AF92BF920F
:1071D000CF92DF92EF92FF92CF93DF93EC01E0E04A
:1071E000DE01AE0FB11D8C91882311F0EF5FF8CF57
:1071F000E150C12CD12C7601812C912C5401839427
:10720000EF3FD1F0DE01AE0FB11DAC9180ED8A0FE2
:107210008A3080F4B0E0D097A50194010E941B3C15
:10722000C60ED71EE81EF91EAAE0B0E00E94103C70
:107230004B015C01E150E4CFC701B601DF91CF9172
:10724000FF90EF90DF90CF90BF90AF909F908F9086
:107250000895F894A895E0E6F0E088E180838BE457
:10726000808378940895F894A89584B7877F84BF25
:10727000E0E6F0E080818861808310827894089550
:10728000FC0180818154823170F48181815482318A
:1072900050F4828180538A3030F4838180538A3065
:1072A00010F480E0089586E008952F923F924F9267
:1072B0005F926F927F928F929F92AF92BF92CF9286
:1072C000DF92EF92FF920F931F93CF93DF93CDB78F
:1072D000DEB7E0970FB6F894DEBF0FBECDBF47E034
:1072E00050E068EE73E08DE694E00E943E3F8091AE
:1072F0006D049FEB980F9A3110F410E009C00E94C2
:10730000D5388111FACF80916D048032B1F315E048
:1073100080916E049FEB980F9A3128F00E94D53827
:10732000811101C015E080916F040E94D538811150
:1073300001C015E0809170049FEB980F9A3118F00E
:10734000803209F015E0809171049FEB980F9A311B
:1073500018F0803209F015E0809172049FEB980FCD
:107360009A3118F0803209F0AAC0111194C18091AD
:107370006D040E940C38282F30E0A4E2B0E00E9497
:10738000FA3B6B017C0180916E040E940C38A701CE
:107390009601280F311D411D511DAAE0B0E00E9449
:1073A000103C6B017C0180916F040E940C38A70196
:1073B0009601280F311D411D511D2BA73CA74DA73C
:1073C0005EA700E714E063E7E62E64E0F62EF8011E
:1073D00081918F010E940C38E82FABE1B0E02BA522
:1073E0003CA54DA55EA50E94103CDC01CB010A978F
:1073F000A109B1099C01AD012E0F311D411D511D87
:107400002BA73CA74DA75EA7E016F10601F745E0C4
:1074100050E06FEE73E08DE694E00E943E3F8DE613
:1074200094E00E944039182F811135C180916D047C
:107430000E940C38082F80916F040E940C38202F76
:1074400030E02A50310946EF4203D001439FB00D8E
:107450001124AD54BF4FA81BB10924EB30E00E94AA
:10746000093C4B015C0180916E040E940C38082F8E
:10747000809170040E940C38202F30E02A5031098E
:107480006AE0629F6001639FD00C11240D2C000CF8
:10749000EE08FF08C80ED11CE11CF11C8C0C9D1CD1
:1074A000AE1CBF1C2091DB032D3358F4822F0E94A9
:1074B000B23B992341F09B7F933019F404C015E04F
:1074C000EAC017E0E8C08091FF039FEF980F9E315C
:1074D00080F480FD0EC080910C0490910D04A09169
:1074E0000E04B0910F04892B8A2B8B2B21F412E010
:1074F000D2C013E0D0C087E0880C991CAA1CBB1C2A
:107500008A95D1F7822F90E0A0E0B0E0805C9F4F99
:10751000AF4FBF4F6C017D01C80CD91CEA1CFB1C8E
:10752000FE017696CE018B965F0111928E179F0712
:10753000E1F7FE013196EFA7F8AB1192AE16BF0648
:10754000E1F74BE1842E912C00E0412C512C3201CB
:107550005FE1252E312C0C3168F48BA59CA5ADA5DF
:10756000BEA5082C04C0B695A795979587950A9453
:10757000D2F713C0023398F48EEE800FA101481B9E
:107580005109CA01A701960104C056954795379540
:1075900027958A95D2F7DA01C901817001C080E090
:1075A000440C551C661C771C480E511C611C711C38
:1075B000C301B20161757375807D927F0E94A63709
:1075C000882329F0602F660FC5010E94CB37C301C5
:1075D000B20167747C738176947E0E94A6378823FB
:1075E00031F0602F660F6F5FC5010E94CB370F5FD0
:1075F00031E0831A9108013509F0ADCF912C812C2F
:1076000097E0E92EF12CCC24C394D12C80E090E0BB
:1076100000E0282D30E0A901082E02C055954795BD
:107620000A94E2F740FF0AC0A701481B590BB601B4
:1076300002C0660F771F4A95E2F7062B0196883045
:10764000910549F7023A60F4692DC5010E94B637E9
:10765000882329F0602F8FA598A90E94CB37939497
:10766000839471EA791590F600E0602F8FA598A9B0
:107670000E94B637F82E602F83E191E00E94B63762
:10768000FF0C4F2D480F602F8DED94E00E94F737CF
:107690000F5F023A51F7812FE0960FB6F894DEBFE4
:1076A0000FBECDBFDF91CF911F910F91FF90EF9053
:1076B000DF90CF90BF90AF909F908F907F906F9012
:1076C0005F904F903F902F900895CF9380912C0220
:1076D000823A90F581110CC060910C0470910D04F8
:1076E00080910E0490910F040E941C2E1092B703FB
:1076F00060912C028DED94E00E94E137C82F0E942A
:10770000812C81E00E940C138BE00E94811660E0C6
:1077100080912C020E94131780E20E948E168C2FFB
:107720000E949A1680E20E948E1680912C028F5F32
:1077300080932C0280E004C080E00E940C1381E062
:10774000CF910895DB018F939F930E94103CBF91CE
:10775000AF91A29F800D911DA39F900DB29F900DA0
:1077600011240895991B79E004C0991F961708F019
:10777000961B881F7A95C9F780950895AA1BBB1B95
:1077800051E107C0AA1FBB1FA617B70710F0A61B21
:10779000B70B881F991F5A95A9F780959095BC0142
:1077A000CD010895A1E21A2EAA1BBB1BFD010DC03D
:1077B000AA1FBB1FEE1FFF1FA217B307E407F507A1
:1077C00020F0A21BB30BE40BF50B661F771F881F7D
:1077D000991F1A9469F760957095809590959B0113
:1077E000AC01BD01CF010895EE0FFF1F0590F4918C
:1077F000E02D0994A29FB001B39FC001A39F700D1B
:10780000811D1124911DB29F700D811D1124911DA8
:1078100008950E94FA3BB7FF0895821B930B0895C9
:107820000E94FA3BA59F900DB49F900DA49F800DE0
:10783000911D11240895B7FF0C94103C0E94103C38
:10784000821B930B08955058BB27AA270E943B3CEC
:107850000C94E53D0E94AC3D38F00E94B33D20F011
:1078600039F49F3F19F426F40C94A93D0EF4E095E9
:10787000E7FB0C94A33DE92F0E940A3E58F3BA1788
:10788000620773078407950720F079F4A6F50C9436
:107890002C3E0EF4E0950B2EBA2FA02D0B01B90152
:1078A00090010C01CA01A0011124FF27591B99F076
:1078B000593F50F4503E68F11A16F040A22F232F82
:1078C000342F4427585FF3CF469537952795A795D2
:1078D000F0405395C9F77EF41F16BA0B620B730B79
:1078E000840BBAF09150A1F0FF0FBB1F661F771FEA
:1078F000881FC2F70EC0BA0F621F731F841F48F49F
:10790000879577956795B795F7959E3F08F0B0CF27
:107910009395880F08F09927EE0F9795879508950E
:107920000E947F3D08F481E008950E94BC3DE395EC
:107930000C94F63D0E94AE3C0C94E53D0E94B33D94
:1079400058F00E94AC3D40F029F45F3F29F00C94C0
:10795000A33D51110C942D3E0C94A93D0E940A3E6A
:1079600068F39923B1F3552391F3951B550BBB276E
:10797000AA2762177307840738F09F5F5F4F220FB3
:10798000331F441FAA1FA9F335D00E2E3AF0E0E8AA
:1079900032D091505040E695001CCAF72BD0FE2FF4
:1079A00029D0660F771F881FBB1F26173707480788
:1079B000AB07B0E809F0BB0B802DBF01FF27935840
:1079C0005F4F3AF09E3F510578F00C94A33D0C9424
:1079D0002D3E5F3FE4F3983ED4F386957795679507
:1079E000B795F7959F5FC9F7880F911D9695879575
:1079F00097F90895E1E0660F771F881FBB1F621794
:107A000073078407BA0720F0621B730B840BBA0B51
:107A1000EE1F88F7E09508950E94133D6894B11118
:107A20000C942D3E08950E94123E88F09F5798F0C6
:107A3000B92F9927B751B0F0E1F0660F771F881F73
:107A4000991F1AF0BA95C9F714C0B13091F00E948D
:107A50002C3EB1E008950C942C3E672F782F882798
:107A6000B85F39F0B93FCCF3869577956795B395B4
:107A7000D9F73EF490958095709561957F4F8F4F23
:107A80009F4F0895E89409C097FB3EF49095809528
:107A9000709561957F4F8F4F9F4F9923A9F0F92FD4
:107AA00096E9BB279395F695879577956795B79552
:107AB000F111F8CFFAF4BB0F11F460FF1BC06F5F38
:107AC0007F4F8F4F9F4F16C0882311F096E911C04A
:107AD000772321F09EE8872F762F05C0662371F06B
:107AE00096E8862F70E060E02AF09A95660F771F7F
:107AF000881FDAF7880F9695879597F90895990F5B
:107B00000008550FAA0BE0E8FEEF16161706E80767
:107B1000F907C0F012161306E407F50798F0621B88
:107B2000730B840B950B39F40A2661F0232B242B5D
:107B3000252B21F408950A2609F4A140A6958FEF7C
:107B4000811D811D089597F99F6780E870E060E0CE
:107B500008959FEF80EC089500240A9416161706E6
:107B600018060906089500240A941216130614062E
:107B7000050608950C94A93D0E94123ED8F3E8949E
:107B8000E0E0BB279F57F0F02AED3FE049EC06C04C
:107B9000EE0FBB0F661F771F881F28F0B23A6207EF
:107BA0007307840728F0B25A620B730B840BE395BA
:107BB0009A9572F7803830F49A95BB0F661F771F3D
:107BC000881FD2F790480C94F03E092E0394000CC5
:107BD00011F4882352F0BB0F40F4BF2B11F460FF67
:107BE00004C06F5F7F4F8F4F9F4F0895EF93E0FF6B
:107BF00007C0A2EA2AED3FE049EC5FEB0E943B3C64
:107C00000E94E53D0F90039401FC9058E8E1F1E0FB
:107C10000C94033F57FD9058440F551F59F05F3F98
:107C200071F04795880F97FB991F61F09F3F79F09E
:107C300087950895121613061406551FF2CF469520
:107C4000F1DF08C0161617061806991FF1CF8695A2
:107C50007105610508940895E894BB276627772786
:107C6000CB0197F908950E94463E0C94E53D0E9491
:107C7000AC3D38F00E94B33D20F0952311F00C94F8
:107C8000A33D0C94A93D11240C942D3E0E940A3E64
:107C900070F3959FC1F3950F50E0551F629FF0015F
:107CA000729FBB27F00DB11D639FAA27F00DB11D78
:107CB000AA1F649F6627B00DA11D661F829F222701
:107CC000B00DA11D621F739FB00DA11D621F839F88
:107CD000A00D611D221F749F3327A00D611D231F5E
:107CE000849F600D211D822F762F6A2F11249F57AC
:107CF00050409AF0F1F088234AF0EE0FFF1FBB1FAF
:107D0000661F771F881F91505040A9F79E3F51056D
:107D100080F00C94A33D0C942D3E5F3FE4F3983E1D
:107D2000D4F3869577956795B795F795E7959F5F17
:107D3000C1F7FE2B880F911D9695879597F90895A9
:107D40009F930E94BC3D0F9007FCEE5F0C94F63DA4
:107D500019F416F40C94A93D0C94EE3E0E94123EC8
:107D6000B8F39923C9F3B6F39F57550B87FF0E94C9
:107D7000FC3E0024A0E640EA900180585695979575
:107D800028F4805C660F771F881F20F026173707BE
:107D9000480730F4621B730B840B202931294A2BCE
:107DA000A69517940794202531254A2758F7660F82
:107DB000771F881F20F026173707480730F4620B1B
:107DC000730B840B200D311D411DA09581F7B90166
:107DD000842F9158880F9695879508959F3F31F08D
:107DE000915020F4879577956795B795880F911DE9
:107DF0009695879597F9089591505040660F771F93
:107E0000881FD2F708959F938F937F936F93FF936B
:107E1000EF939B01AC010E94333EEF91FF910E94D2
:107E2000173F2F913F914F915F910C94333EDF9319
:107E3000CF931F930F93FF92EF92DF927B018C0100
:107E4000689406C0DA2EEF010E94463EFE01E894D7
:107E5000A5912591359145915591A6F3EF010E9489
:107E60003B3CFE019701A801DA9469F7DF90EF909F
:107E7000FF900F911F91CF91DF910895DC01CB010D
:107E8000FC01F999FECF06C0F2BDE1BDF89A31962A
:107E900000B40D9241505040B8F70895F999FECFC3
:107EA00092BD81BDF89A992780B50895A6E1B0E00A
:107EB00044E050E00C94403FDC01CB0103C02D9125
:107EC0000E94673F41505040D0F70895262FF999FE
:107ED000FECF1FBA92BD81BD20BD0FB6F894FA9AAD
:107EE000F99A0FBE01960895242F0E94673F252F0F
:107EF0000E94673F0C947C3F0E94663F272F0C94A2
:067F0000673FF894FFCF7B
:107F06000A000A000000404200C03B4400CC3B4649
:107F1600060A80C08E25E02502CD1A1AA92C6A20F1
:107F260093B34705301AC600DFCFC7C3C1C0D0D848
:107F3600DCDEF9E8EAF4FCE2F6E0F8E7F5E4FBFA61
:107F4600F7E6EDF2F0FDF1E1F3E9EBECEFD2D18CDF
:107F560095B33244003344004E6F002D2D002D2082
:107F6600732D00524D430047534100474741004798
:107F7600535600100E080A0609090D06000A8096D7
:107F86009840420FA08601102700E80300F4010084
:107F96006400000A0000A400A800AC00B000540071
:107FA6005800A0009F00B800BC00C400C5008C00AB
:107FB600F50300004C004D00740060006400E80307
:107FC600EF0368009000940098009C009D009E00BE
:107FD60002005C004E006C00C7004F008700B40032
:107FE6007800F40303007C008000840048008500CC
:047FF6000100500036
:00000001FF
